:020000041100E9
:10300000F7B5164B0192C318021D002000938823C8
:103010005B05D3181B685C1C1AD09CB2402C18D8D6
:103020008D781E0CAC466746CD782D023D43AE42EE
:1030300006D1019800280ED110000C70240A4C70A3
:1030400003249BB20733A343D218009B9A42DED3DA
:10305000FEBD4432F9E71000FAE7C046FC0F00005D
:10306000802213B503000324019189B25201073174
:103070009B18A14304305A1A88235B05C3181B68A8
:10308000591C03D190429241104016BD99B240297B
:1030900007D80B000733A343C0189042ECD300209D
:1030A000F3E74430F9E7134B134A1B68126810B575
:1030B000FA24934201D81A00F824104BE4021B684A
:1030C0009A4210D813000E4A12689A420ED3013366
:1030D00007D1F823DB029C4203D10A49054808F0D6
:1030E0003BFA200010BDFC24E402ECE7FE24E402DD
:1030F000F7E7C04600C0071100D0071100E0071134
:1031000000F00711FFFFFF7FF0B59BB015000490A2
:103110000391402A00D9A0E006AB59801A80FFF73E
:10312000C2FF0400042816D9002206A9FFF768FF91
:10313000052810D906AB1B88AB420CD1002D07D057
:10314000514B2A000499C01808F0EEF8002802D16B
:1031500001201BB0F0BD06AB1D8020000699FFF7D3
:103160007FFF041E7BD1069B0793FFF79CFF802304
:103170005B01C618802307001B039E4201D3F8267B
:10318000F60288235B05F31801931B68013302D014
:10319000019808F019F93D49019808F0DDF93B1D47
:1031A0000293331D05938822029B52059B181B68CE
:1031B00008935A1C3CD044219AB20091402A04D86A
:1031C0000320D11D814389B2009103991B0C8B42CE
:1031D00024D0402A22D80122300008A9FFF710FF8E
:1031E000021E1BD1380008A9FFF70AFF04000428BB
:1031F00031D9009A059B9B1880225201B218934244
:1032000040D288235B05C118009A09A807F0B4FFD3
:103210001D4B009A09A9F01807F06EFF009A029B57
:103220009446634402931A4B029AFB189A42BAD30B
:1032300088235B05FC1821680198013908F08CF996
:10324000200008F0C1F8039A07AB5A8030000799B4
:10325000FFF706FF0400002C03D1002079E70428C3
:10326000FBD988235B05E018069908F075F903235C
:10327000EA1C9A4300D16BE7034B0499E01807F06E
:103280003BFF65E70424ECE704000011FFFFFF7F2C
:10329000F80F0000F7B505001400402A21D80027D8
:1032A00001AE71803780FFF7FEFE042816D93A0080
:1032B0003100FFF7A5FE042810D93688BC420BD098
:1032C000BD4209D0221CB44200D9321C064B92B236
:1032D000C118280007F050FF30B2FEBDC04300B255
:1032E000FBE703204042F8E70400001137B5042251
:1032F00004000D0001A81649FFF7CCFF02000428C6
:103300000BD1019BA34208D3AB4204D0104901A8C2
:103310000195FFF7F9FE01203EBD0E4C2368200009
:10332000019308F051F8019920000139019108F04A
:1033300013F980235B01E418074B9C42EED1042271
:10334000034901A80195FFF7DFFE0020E4E7C0462E
:103350005555000000C007110000081130B589B0B4
:1033600008F062F810226946254808F0EDF8254B70
:10337000009A9A420ED1019B029A0F2B33D800215A
:1033800001240698013B08D2002900D00292029B3A
:10339000013331D10023029325E0551CF2D1020004
:1033A0002100EFE710341022200004A908F0CCF827
:1033B000029B013301D1069B0293882304995B058C
:1033C000C918059B06981A03120B049105928142B5
:1033D00003D02B4201D107F0CFFE019B013B0193AB
:1033E000019B002BDED1029B002B03D00493049899
:1033F0004168084709B030BDE025014C2D03EFE7D7
:1034000000000111504859368022F8B5964C974B70
:10341000D200002120001C6008F046F82300944AE6
:1034200088331A60934B1A786A23002A00D011332C
:10343000E3620A232365904B37221B780820A3639D
:103440008E4B2118E361102323628D4B3B25636172
:10345000C823DB00A36123008C331A602823013AC0
:10346000E26320646364CA67043A211DCA672100CD
:10347000BC310D602100C03108602100C4310B60F7
:1034800021000635CC310D602100083DC8310D60AA
:103490002100D0310A602200D43210602200D832DC
:1034A000136022000227E032210017604222DC3143
:1034B0000A6021001B3DE4310D602100E831086005
:1034C0002100EC310B6023000521F4331960230047
:1034D000F0331A602300183290331A6023009433BB
:1034E000186023001E3A98331A60AF23DB00236074
:1034F000644BFA262363644B644DE360644BF03104
:10350000A3642300FF31FC33B600A16021611E607B
:10351000A5627325E5656D3D6565A56596255D4AE2
:10352000AD00E264666258606766A56600270925FB
:10353000A767E566584F594D606720002567E26729
:103540003A6015279C30676007001A203860200019
:10355000A0300700212038602000A83007004C4828
:1035600038602000F830066026006427A4363760F3
:1035700026005F3FAC3637602600033FB036376029
:103580002600C637B436376026000027B8363760C5
:1035900038269E60424E96205E64424E5A66DE6138
:1035A000414E9A645E62F53EFF3E9E621E269A6719
:1035B000354A8000DE661F675F67DD651D6618623D
:1035C000DA67BE23394A5B00E250394BD8382350C2
:1035D00004302250C4225200A350C623E4205B00D2
:1035E000E1500433334AE1503349344BD16034491C
:1035F000800019503349E938FF38195032490430F6
:10360000195032493248D16132491163324951630C
:103610001900F4310860CE20304940001160304973
:10362000195019002F48F83108602F49D1658221BF
:103630002E4A89005A501A002D490832D1671A00C3
:103640002C49B432116088212B4A89005A501A0043
:103650002A49883211602A4ADA6407F0EDFC012019
:1036600007F0AAFEF8BDC0460004FF1F3464FF1F28
:10367000006FFF1F1044FF1F4A0AFF1F3A07000098
:1036800080C3C9019A020000DC0500006A1800002E
:1036900050C3000088130000F009FF1F204E0000F7
:1036A0006509FF1F68100000C409000040420F00B8
:1036B00010270000FC00FF1F751CFF1F0000FF1FEC
:1036C000C92CFF1F5130FF1FE92EFF1F3520FF1FA0
:1036D0002527FF1F5120FF1FFD21FF1FC11FFF1FB7
:1036E0004929FF1F312AFF1F8D19FF1F5528FF1F72
:1036F0007925FF1F8525FF1FC11EFF1F791FFF1F93
:10370000391EFF1F0223F0B50124634D634E2B7059
:10371000634B8BB01C70634F039333680021092007
:10372000BB7006F021FB092006F028FA031E05D124
:10373000BA78552A02D0332A00D0A1E000233360A2
:10374000042006F06FFC07F097FEFFF75DFE07F020
:10375000ABFC0D220124544B1E261A700022534B41
:103760001C70534B1A70534B1F3219689143163A11
:103770000A431A60602219689143403A0A431A606A
:1037800007F032FC07F0D8FD4B4B9847C120FF21D2
:103790004A4B80001A588A431A50C5229200985802
:1037A0008843BF39014399509858454908408021C2
:1037B000C9010143802099509958C0050902090A9E
:1037C0000143995080213F48490107F09DFE0323A2
:1037D000220000933C4901943C4807F05DFE16220C
:1037E0003B4904A807F0C8FC02AB04ACF6186178AA
:1037F0002078023406F0D2F9A642F8D1354C0320E5
:10380000012106F0DFFA2268334B03201A40A0237F
:10381000DB0213432360802322689B04134323604D
:1038200022682E4B1A4080239B03134323602C4AAB
:103830002C4B934200D8012007F03EFC07F0CCFD52
:1038400080232268DB0413432360287807F054FEAA
:10385000039B1878C0B207F03FFC07F005FE224931
:10386000042007F069FB06F0A9FB00F03FF800F028
:1038700077FD00F01FFE00F0A1FB00200BB0F0BDB3
:1038800000902100184A042007F0F6FC8023DB0595
:103890009C62FFF763FD53E74A0AFF1F34F00040C4
:1038A0001044FF1FDC61FF1F480AFF1F490AFF1F6A
:1038B000680AFF1FBCF00040E1A2000000E100E048
:1038C000FF00FFFF1444FF1F9856FF1F1454FF1FF3
:1038D00088B5001114F00040FF7FF8FFFFFF9FFF45
:1038E0000080FF1F006FFF1F3B000108002210B582
:1038F0001100112007F090FC10BD0000F8B5002366
:103900000926374F374C3B62E3681120B343E3602D
:1039100007F0A2FD112007F04FFB112007F004FB78
:103920004023226880251343236080236268DB02E2
:1039300013436360A3682C4A2B43A360A36802214E
:103940001340A3608023A2689B0113431022A3604D
:10395000236C072093432364236C0F3A134323649F
:1039600080235B003B62226B204B1A402263626B18
:103970001A406263A26B1A40A263E26B1340E363D6
:10398000E3681B4A1340E36006F008F901210720B1
:1039900006F018FA174B11205A6C15435D6407F0B6
:1039A000C3FBFD21144B154A89005A508023C720C0
:1039B000626B5B0313436363E36880003343E3603C
:1039C0000F4B104A19581140802212020A431A5014
:1039D000802292051A6008220B4B5A63F8BDC0463C
:1039E00000F000403CF00040FFFFDFFFEFFFEFFF83
:1039F000FFFF7FFF003800400000FF1F5118FF1F2E
:103A000000E100E0FF00FFFF0000054007B50422D1
:103A1000044901A807F0B0FB012101A807F0ACFCA4
:103A200007BDC0469EB5001170B52B4C238C002BF2
:103A30002AD0FA22D200934201D2FFF7E7FF228A6E
:103A4000238C002A21D1DA0023826382A382E382BD
:103A500023836383A383E38322606260A260E260C6
:103A60001E4D1F4A64206B8093420AD8FA22002020
:103A7000D200934205D91B4A0A21981807F04CFB43
:103A8000C0B200232871238470BD0720E11CCA7FC7
:103A900001320240CA7705D10325201DC17F0131C3
:103AA0002940C17708325200A352002321001A0096
:103AB000088A01321B180231082AF9D1221DD27F4F
:103AC0009200A350626823689B18A2689B18E26862
:103AD0009B185B099BB2C3E71061FF1FC061FF1F0A
:103AE000B70B000030F8FFFF30B503A804880B20A7
:103AF000002C0ED14968074D087849780902014326
:103B00000A20A94205D1012120001980024B1B790E
:103B1000137030BD192A0000C061FF1FF7B51500F2
:103B200008AA16884A680F4F147852781202224366
:103B30000A24BA4214D10122DBB2019200962A0073
:103B400007F08CF9041E0BD1074B1B68002B07D024
:103B500068782A7800021043424250410130984769
:103B60002000FEBD022900003C61FF1F30B5012589
:103B700003790400BFB02B4211D00A49408806F0F7
:103B8000D9FC28420BD0084B01A95B8D4D800B80DE
:103B9000064B00221B7960880B7103F0D7FD3FB004
:103BA00030BDC0463461FF1FD040FF1FC061FF1F02
:103BB00010B50549054806F073FC0421044A054880
:103BC00006F030FC10BDC0463461FF1FFFFF00004F
:103BD000A4B50011D040FF1F10B5024804F038FC16
:103BE00010BDC0466D3B0011F0B593B005921D00AD
:103BF000DAB20F239B1ADFB20E239B1ADBB20493B7
:103C00001C9B049A023B5B08DB00134306AA13705B
:103C1000199E06AB2A0003900191581C059907F0E4
:103C2000ABFA3400002206AB013BBA4252D1002C61
:103C300000D0B9E0102221000AA807F035FC0AAB39
:103C4000029306A91A78615C01344A401A70013364
:103C5000102CF6D10AAA1100019807F03DFC202291
:103C6000212006AB9B18049A05991A7006AB2A000E
:103C7000C01807F081FA01350EAB58193A0000213F
:103C800007F012FC2F210123250006AA52181370F9
:103C9000002E24D112AB3A003100D81B07F004FCEF
:103CA000019806AA0EA907F017FC029B06AA925DCE
:103CB0001B7801365340029A1370130001330293AC
:103CC000102EF2D11C9A1B980AA907F055FA002071
:103CD00013B0F0BD01321C74D2B2240AA4E7340040
:103CE000102E00D92C00039B002B19D119002A009B
:103CF00006A807F0D9FB2200189906A807F03CFA9D
:103D0000039B0AAA06A81178185C01334140117080
:103D10000132102BF6D10AAA1100019807F0DCFB42
:103D2000019806AA0EA907F0D7FB0023189A06A946
:103D3000C95CD25C4A401A99CA5401339C42F5D1FD
:103D4000039B012B19D11022002106A807F0ACFB20
:103D500022001A9906A807F00FFA00230AAA06A85B
:103D60001178185C0133414011700132102BF6D1EB
:103D70000AAA1100019807F0AFFB00221A9B361B1C
:103D80001B191A93189B0EA91B191893BA4200D13C
:103D90007EE7CB7B01390133DBB20B74002B00D003
:103DA00076E70132D2B2F1E70120404290E700000D
:103DB00010B5134A134B5179134C19701179200027
:103DC0005970D17899709178D970517812781971A9
:103DD0005A712E2252429A712A32DA7145321A727F
:103DE0000A49313AFFF756FA102808D0102120006E
:103DF00007F0BAFA102220000449FFF785F910BD38
:103E00006509FF1F5061FF1F4061FF1F0DBC0000CF
:103E1000F0B5431805000020114F124A3E8889B0C2
:103E20000C00114956720792320A4A70320ECA705B
:103E300088701E70042639889870090A5970D870E5
:103E40009B19039301940D230849079A0496029540
:103E50000095FFF7C9FE0834E0B209B0F0BDC046D6
:103E6000C061FF1F5061FF1F5961FF1F4061FF1FAD
:103E7000012202700C4A0300117941700C209870E5
:103E80009178D970D17819713A21597192799A71D2
:103E90003E22DA71054A117B1972517B5972917B6E
:103EA000D27B9972DA727047C061FF1FC861FF1F31
:103EB0003A230370074B9B7943703E238370064B74
:103EC000197BC170597B0171997BDB7B41718371D7
:103ED00007207047C061FF1FC861FF1F022370B534
:103EE0000370013B43701C4A053383701033037128
:103EF0001168443B43712A33837104002022080077
:103F0000164B1040DB7C114215D0250021320835BC
:103F10002800E271002B0BD0FFF7CAFF0100280038
:103F2000FFF776FF0430C0B2E0700430C0B270BD5D
:103F3000FFF79EFFF2E7402220722000E271084A5C
:103F40000A3012886272002B03D0FFF7B1FF0630EF
:103F5000E9E7FFF78DFFFAE7E061FF1FC861FF1F88
:103F6000C061FF1F10B5142007F0F6F8124B1422A1
:103F70000021186007F098FA002007F05DFA012090
:103F800007F022F8022007F047FA032003F004FDAF
:103F9000042005F019FD052002F042FF062003F081
:103FA0000FFC072001F054F8082006F01BFA092046
:103FB00000F0E6FD10BDC0466061FF1F06F0C4FFC3
:103FC000012007F019F907F047F80000094B10B578
:103FD0000400984205D0012904D12000064906F0CA
:103FE0005FFA10BD0229FCD1013904F0EFF9002875
:103FF000F3D0F6E7FEFF00008661FF1F70B50D7A73
:10400000100004AA2C00168810221440154220D15A
:10401000002E20D10A78022A18D14A6851781578E2
:104020000E4A09022943914205D00D4A914209D016
:104030001C800A2404E014220A491A8007F09CF824
:10404000200070BD0C2208491A80F7E71C8001246B
:10405000F6E70824F4E70B24F2E7C046F3FF00007C
:10406000F4FF00009C42FF1F5CB6001110B5040075
:104070000749084806F014FA074804F029F9002017
:10408000E40704D50721054A054806F0CBF910BD21
:104090008661FF1FFFFF0000CD3F0011E8B5001152
:1040A0001441FF1F00B50C4BBFB01A780B4902A892
:1040B00000F0A4FA6B4680B2D880002809D06A4686
:1040C000074B01A91B889380064B0022188803F038
:1040D0003DFB3FB000BDC0466461FF1F6561FF1F2F
:1040E0006E41FF1F7042FF1F00B50C4BBFB01A7826
:1040F0000B4902A801F070FA6B4680B2D880002804
:1041000009D06A46074B01A95B8D9380064B0022BC
:10411000188803F01BFB3FB000BDC0468E61FF1F37
:104120008F61FF1F1441FF1F7042FF1FF7B50E0084
:10413000377A1C0008AB11003D001A8820231D406F
:104140001F423CD13378022B3BD173681F785B78D8
:104150001B023B431E4FBB4208D01E4FBB4214D034
:104160001D4DAB4221D00A252800FEBD002A2AD1D0
:10417000142C2AD82200F06806F0FEFF174B1C70A2
:10418000012CF1D9FFF7B0FFEEE7002A1BD1202C5C
:104190001BD82200F06806F0EFFF114B04211C70C1
:1041A000104B187807F0D8F8DEE7E3B2012400924C
:1041B00001940A00310006F051FE0500D4E70825FD
:1041C000D2E70125D0E70B25CEE70D25CCE7C04689
:1041D000F3FF0000F4FF0000022900008E61FF1FC2
:1041E0006461FF1FFC61FF1F332310B504000370DF
:1041F00005220749013006F0BFFF064B0A201B6865
:104200001A0AA371E2711A0C1B0E2272637210BD9E
:10421000C061FF1FEC61FF1F30B501250379040069
:10422000BFB02B4213D00B49408806F083F92842D7
:104230000DD06A46084B02A81B889380FFF7D4FF75
:104240006B46D8800022608801A903F07FFA3FB056
:1042500030BDC0468661FF1F6E41FF1F10B502488A
:1042600004F0F6F810BDC0461942001170B51600F2
:1042700004AA148805AA15784A68507811780002B3
:104280002A4A0843801805284BD806F075FE031308
:104290001E29343F0720022C0BD80322121BAA42EE
:1042A00000D92A0022491A803000091906F064FF5B
:1042B000002070BD0720112CFBD81222121BAA422D
:1042C00000D92A001B491A80EEE707200E2CF0D8EF
:1042D0000F22121BAA4200D92A0017491A80E3E7CD
:1042E0000720032CE5D80422121BAA4200D92A0079
:1042F00012491A80D8E70720032CDAD80422121BAF
:10430000AA4200D92A000E491A80CDE70720022CC4
:10431000CFD80322121BAA4200D92A0009491A80C9
:10432000C2E700220A201A80C3E7C046DCD5FFFF9F
:1043300032B60011AC61FF1F22B600111DB600118C
:1043400018B6001114B6001110B50D21024A034829
:1043500006F068F810BDC04608B600118441FF1F82
:1043600010B5084CE368002B08D18022064B52029E
:104370001B689B186360054B1B68236007F0D4F82B
:10438000A06010BDEC61FF1FC8F00040CCF0004001
:1043900070B5184A936A916A9942FBD116498A68A6
:1043A0009A421FD39A1A8B60144B0126186893B255
:1043B000D202D20E4343424300204C681B0A1B1911
:1043C00012029B180E4C0A684B60551CA3420CD875
:1043D000002801D04B600A600A4A136008680A4B43
:1043E000186070BD581E821ADDE7084A30009B181D
:1043F0002A00EAE700F00040EC61FF1F140AFF1FEB
:1044000040420F00C8F00040CCF00040C0BDF0FFBB
:1044100070B51F4C23793F2B01D93F2323711D4BCE
:1044200022791A701878C0B206F0F6FD18231A49DE
:104430001A4A0B801A4913800B805380A3791949BB
:1044400080200B800C21938001334B43164D191CA7
:104450000001834200D9011C2980D1806379002B9F
:1044600011D101336371237A012B01D80223237206
:104470006279237A0D4853430A21584306F04CFED3
:104480000B4D286070BDA02BEDD9A023EAE7C046F4
:10449000E061FF1F480AFF1F6E42FF1FBC43FF1F62
:1044A0006C42FF1F6A42FF1F6842FF1F710200003B
:1044B000C861FF1F70B520210020FEF717FF084CD0
:1044C000002805D1074B23CB23C4FFF7A1FF70BD04
:1044D0000C2220000449FEF7DDFE0C28F2D1F4E79F
:1044E000E061FF1F50B60011FC0C0000F0B51D4C40
:1044F0008022A5440400882069465201400506F048
:104500002BFD902212016A441300200032C832C3EE
:1045100016C816C38023144C144FA6689B0333435C
:10452000A3603B6006F0B0FD8823A0685B05C0185F
:1045300006F04AFF0025882329008022A0685B0539
:10454000C01840196944520006F0D6FD8023013599
:10455000FF355B019D42EED1A6603E60044B9D4459
:10456000F0BDC046FCEFFFFF2C43FF1F9808FF1F64
:1045700004100000F0B5040087B0002825D068467C
:1045800006F0A2FE1B4C022806D106226946200036
:1045900006F0CAFE002816D06946002301250F2622
:1045A0002F00E25C013310091030874038002F00E3
:1045B000324097403A0002434A610439062BEFD15A
:1045C0006846FFF793FF07B0F0BD182269460A4816
:1045D00006F0C2FC6A46A300D358013305D0182266
:1045E000FF21684606F060FFEAE70134062CF1D1AE
:1045F000E9E7C0466509FF1F00090011F0B5002674
:1046000004000D0085B0B24200D19BE00B78A87881
:1046100001310191697800020843E9782F79090492
:1046200001433F060F43039723706670232B00D18D
:10463000DFE042D8102B00D1ECE01DD8062B00D1D2
:10464000BAE0072B00D1B0E0B34275D0012B19D1ED
:10465000931E994F132B07D86B78002B00D0FFE0E7
:1046600000F0FCF900F032FA944B39001E78601C1F
:10467000721E06F081FD65E0112B00D1EAE0182BD7
:1046800000D16AE0DB2B00D0F6E0042A00D888E0F5
:104690001026052A05D0561F32003800691D06F085
:1046A0006BFD05222900200006F066FD320039006E
:1046B000601D06F061FD053644E0562B47D01CD83E
:1046C000332B00D190E0552BDCD1013A7C4D0C2AE4
:1046D0003BD8002A0AD02800019906F04DFDFFF7CB
:1046E00097FE0C2228007749FEF70EFD0C222900C8
:1046F000601C06F041FD0D2624E0712B63D0722B67
:1047000069D0DC2BBED1022A4BD96B78BFB2637063
:10471000AB78A370032A05D0033A390092B2E81CA3
:10472000FEF7F2FC10223900E01CFEF7B3FDC61CB8
:10473000002807DA607036E00C222000624906F09B
:104740001BFD0C26300005B0F0BD0C22C3E75C4D0C
:104750005E4B2A0043CB43C2C1E75D4D112A12D103
:1047600028000199013A06F0DFFD00280BD0102245
:104770000199280006F000FD102256492800FEF796
:10478000C3FCFFF715FB102228005249FEF782FDFB
:104790000200102805D12900601C06F0EDFC11264E
:1047A000D0E7FF2363700226CCE712224A49601C3F
:1047B00006F0E2FC1326C5E708224849601C06F013
:1047C000DBFC0926BEE76978F029EAD8444B188853
:1047D00001F05EFBE7E7434B012A03D06A785A7089
:1047E0006270E0E75B78DDE72000FFF7FDFC060084
:1047F000A8E7042A04D93C4D2F6006F095FEA86076
:10480000FFF7C6FD0422039003A9601C06F0B4FC68
:10481000052697E7354D062A15D906222800019965
:1048200006F082FD00280ED006220199280006F02D
:10483000A3FC06222E492800FEF766FC0123294A24
:1048400051780B43537006222900601C06F094FC3B
:10485000072677E7012AA4D06878FFF78BFEA2E746
:10486000551E2A000199380006F086FC38002149BF
:10487000AAB2FEF749FCF5E6DA2B92D1042A90D9C8
:10488000082A15D9AB796A791B021343EA79120415
:104890001A432B7A1B0613433B603B680522290011
:1048A0002000039306F068FC0422601D03A986E73C
:1048B000FE236370F1E7C046DD63FF1FDB63FF1F6C
:1048C000E061FF1FFC0C00005CB6001150B6001147
:1048D0004061FF1F0DBC0000AC61FF1F3043FF1F94
:1048E0007042FF1FDC61FF1FEC61FF1F6509FF1FA6
:1048F000ADAC0000AEDE000070470000020010B555
:10490000094B0A32094C92B2DA815A829881188294
:10491000207802F023F90422054B012120781A7037
:1049200006F01AFD10BDC046BA42FF1F2664FF1FE5
:104930002564FF1F013870B5042809D806F01CFB58
:10494000030927081200204B0221187806F004FD05
:1049500070BD1D4B0821187806F02EFC00221B4B61
:104960001A74F5E780220024184B52001A82FA22AA
:10497000DC74174B144D5B7A920008215A43287857
:1049800006F09AFD2100287806F0BEFCE0E70E4B09
:104990000821187806F010FC0E48FFF79FFA0C4B20
:1049A0000D4A9B7993800D4A13800022074BDA74DD
:1049B0000132FF321A820A4B5B78002BC8D0094AB9
:1049C000136006F081FDC3E7FC61FF1FC861FF1F94
:1049D000E061FF1F7942FF1FBC43FF1F6A42FF1FB8
:1049E000DC61FF1F34F0004010B5002909D109280F
:1049F00007D1063805F0E6F9024B8021187806F059
:104A0000ABFC10BDFC61FF1F10B5012909D10928BD
:104A100007D1063805F0D6F9024B8021187806F048
:104A20009BFC10BDFC61FF1F0300F0B50A4D8E1802
:104A3000B14202D152008018F0BD0C782F682409D1
:104A40003C5D0F271C700C7801313C402F683C5DA9
:104A50005C700233ECE7C0466442FF1F0C22124B2D
:104A600010B51A700B23114C11492370093A023BFF
:104A70001048637006F080FB2D2301220E490F4879
:104A80006371FFF7D1FF01220D49FFF7CDFF01222E
:104A90000C49FFF7C9FF030000200B490200187002
:104AA000FEF732FB10BDC046FA63FF1FDB63FF1F3A
:104AB00032B60011DD63FF1F6709FF1FE163FF1FAF
:104AC0006609FF1F6509FF1FAEDE000070B5134CBD
:104AD000142220001249FEF7DDFB431E114D132B5B
:104AE00019D8AB78002B16D0431C2B7009236B70A0
:104AF00000230019037028780B4B01302900C0B245
:104B0000187006F031FB297822000139C9B2002063
:104B100005F0A6FB70BDFFF7A1FFECE7DD63FF1F0B
:104B2000AEDE0000DB63FF1FFA63FF1F10B5114B01
:104B30001A781870002A0ED000280BD10E4B1A7864
:104B4000062A07D85423D340DB0703D50B4B18782C
:104B500002F004F810BD0028FCD0074B1B78012B95
:104B600002D0033B022BF5D8044B0121187806F044
:104B7000F3FBEFE7FE63FF1F2564FF1F2664FF1FA3
:104B800070B54F4E4F4A50493070092005F0F4F986
:104B90000121032005F016F9032005F0DBF906F0EA
:104BA00023FB032249494A48FFF73EFF2D24030017
:104BB00088211C70042249050130FFF735FF30239E
:104BC0000470444D444C437083702E3B06222000F9
:104BD0004249EB87FEF75EFB062813D0200006F063
:104BE00073FB022809D00321200006F0BDFB8D23B2
:104BF000E3706E3B2371193363710622200037493D
:104C0000FEF782FA364B1B68FC335C64FFF75EFFED
:104C1000FFF7CEF80020FFF789FF324C324A01211E
:104C2000324B1278207801F05BFF314A314B127819
:104C30002078002101F054FF01222F4B2F4C1A70D5
:104C40002F4B9B78552B33D1193B63742D4A2E4B38
:104C5000AB81EA812B826A822021307806F084FCC5
:104C60000120404205F048FB0120404205F0E4FBF2
:104C7000FFF76AFBFEF79CFF01204042FFF7F6F9C1
:104C8000012006F089FAF02001F0E6F801213078E1
:104C900006F062FB307802F0BDF81C4806F0B4FA6A
:104CA000FEF72CFE1A4B1B4A9B689B18A36070BD35
:104CB0006422194B5B7953431A000A32C8E7C04695
:104CC000FC61FF1FE9490011094A00113043FF1F31
:104CD000AC61FF1FBA42FF1F6509FF1FADAC0000AA
:104CE0003464FF1F2664FF1F9842FF1F7942FF1F95
:104CF000FA63FF1FDB63FF1FCC63FF1FC861FF1F49
:104D0000DC61FF1FCE090000C4090000FE61FF1F27
:104D1000EC61FF1F0000B8FCE061FF1FF8B50A005E
:104D200020230D001A40194200D16BE07A4B1B780A
:104D3000002B3DD0FFF72CFB784B794C794E9968CE
:104D40006268737A8A1ADB039A4234D36160FEF791
:104D5000D5FD637C002B28D0013BDBB26374002BB4
:104D600023D1714B9B78552B01D106F0ADFBE37C31
:104D70006E4F002B32D010236374BB79002B14D1FB
:104D8000A27C002A02D0A374FEF74EFE3B88684E38
:104D9000013330003B80FFF7A1F8310006F0ACFA98
:104DA00000237820E374FFF7A9FD237C01332374EB
:104DB00020206840F8BDA37C002BCAD00023A37438
:104DC000FEF732FE594A5A4F1388380001331380D8
:104DD000FFF784F8390006F08FFABAE7A27C002AC0
:104DE00002D0A374FEF720FE3B8801333B80504F76
:104DF0003800FFF773F8390006F07EFA6423707903
:104E00005843D0E70BB2002B0ADA4A4B187806F069
:104E100093FB002801D006F0DFF980200002C8E7EC
:104E20000224214206D03E4B01201A74FFF77EFE79
:104E30002000BEE70824214204D0FFF7A9FAFEF7BC
:104E40005DFDF5E710230E001E4019420FD0FEF75E
:104E5000EBFD314B1B78002B07D1FEF7BDFE314B2C
:104E60001B68DB0701D5FFF7F9F91020A1E7012442
:104E7000214209D0304800F0AFF806F00DF93100BA
:104E8000032004F09FFFD3E70B063BD5092004F075
:104E900075FE264B5A79002827D0224203D02243A0
:104EA0005A71802085E71E4922435A711A4AC86800
:104EB00012780130C8609C71002A1AD01A881C4CE4
:104EC00001321A800123CB740F334B74134B1B4AEE
:104ED0009B6820009B188B60FFF700F8210006F00C
:104EE0000BFA7820FFF70AFDDBE7A2435A719871AD
:104EF000D7E70C4B1B68DB07D3D5FFF749FAFFF761
:104F0000ADF9CEE7042408002040214200D151E74A
:104F1000FFF7C8F88CE7C046FE63FF1FEC61FF1F78
:104F2000C861FF1FE061FF1FDC61FF1FC061FF1F41
:104F30007942FF1FFC61FF1F5C42FF1F000082FCE3
:104F4000F0B51B4B1B4F1B883A8804001A4E1B4DB3
:104F500085B09A420DD832889A420AD3184B1A88E3
:104F60002B889A4205D1174A174B12881B889A4200
:104F70001BD0052000F0C6FF3B8802AA13803388AF
:104F8000019053802B88114D93800F4B02A91B88F1
:104F9000D3800F4B2A78188802F0E2FC0D4B0821D1
:104FA0002878019A1C7006F0EFF905B0F0BDC046F4
:104FB000CA63FF1F6E42FF1F6C42FF1F6A42FF1F42
:104FC000C863FF1FC663FF1F6842FF1F2664FF1FE1
:104FD0007042FF1FC463FF1F13B50C4B1C78002CDD
:104FE00011D1002801D00A4B18600A4A0A4B1178E7
:104FF0000A4A10780A4A01920A4A0092002205F0F1
:1050000027F8200016BD1124FBE7C0462564FF1FCA
:10501000C063FF1F2464FF1F1464FF1F2664FF1F6B
:105020000064FF1F0464FF1F10B5064B12201B789D
:10503000052B06D1044B13221988044B187801F074
:105040003DF910BD2564FF1F7042FF1F2664FF1F3E
:1050500010B500240122114B52421870104B1C70E5
:10506000104B1A8001F0D6FE04220F4B21001A705B
:105070000E480C3205F088FF102221000C4805F084
:1050800083FF07220B4B1C600B4B1C700B4B1C70DF
:105090000B4B1A700B4B1C7010BDC0462664FF1FD3
:1050A0002564FF1F7042FF1F2464FF1F1464FF1F4D
:1050B0000464FF1F0064FF1FDA63FF1FD963FF1F33
:1050C0007242FF1FD863FF1FF8B5174C0600257802
:1050D00006A814240078052D23D1B41F134FA5B2C0
:1050E0001824BD421DD88D1FADB2BD4219D8FA2576
:1050F0006D00AA4215D21D000D4F0A3DADB2BD4252
:105100000FD80C4C26800C4C21800C4900240A80BE
:105110000B4A1380FFF714FF0A4B0421187806F09E
:105120004BF82000F8BDC0462564FF1F790C000035
:10513000750C00006E42FF1F6C42FF1F6A42FF1F8A
:105140006842FF1F2664FF1FF0B50BB20D0089B047
:10515000002B00DB70E1A44E307806F0EDF9041E60
:1051600050D00378A22B00D122E1D02B1AD0912B62
:1051700045D143780E2B42D19C4B82889A423ED136
:105180009B4A83681278052A39D1032018567F2854
:1051900035D0984B1B68002B31D05B68002B2ED08C
:1051A00098472CE08078072829D805F0E5FE0428E8
:1051B000183F3F74A8D86378002B0CD101218C4B89
:1051C00019708D4B1A78002A5BD08C4B307801F027
:1051D00087FC002855D00722854B1A7051E0617872
:1051E0000029F8D1E378002B11D0854A854B12783D
:1051F000307801F075FC60706378002BEBD12000F3
:1052000005F0EAFF80200002684009B0F0BD784B4D
:105210001B78022BF3D00121307805F0EDFE002839
:10522000EAD10121307806F097F8E5E76378002BA2
:10523000D1D16F4F032807D13B78052B02D1013321
:105240003B701EE00223FBE76F4B1A886F4B029303
:10525000002A0BD01B78002B03D00121307806F0F8
:1052600093F83B78062B04D1013BE9E7029B1A70C7
:10527000F7E7042B41D10121029B3078197006F029
:105280006BF85C4B1B68002BB9D01B68002BB6D0A9
:10529000574A107884E76378554F002B27D10622B0
:1052A000211D5B4805F068FF62895A4B5A491A80F4
:1052B000A2895A4B1A80E3890B800521397058491D
:1052C0000A80584A1380228A574B1A80574B1B7802
:1052D000012B09D11F2000F015FEFA229200424353
:1052E0000421307806F050F80022484B75E7312B46
:1052F00000D070E70022454B1A700323A0E7062276
:105300000021434805F040FE0023454A0421138054
:10531000444A30781380444A138005F04DFF082139
:10532000307805F049FFA379083B5A425341304A8F
:1053300003331370304B1B78002B06D0334B30787F
:105340001A78002A06D001F009FC0122314B5242A2
:105350001A8096E70121197005F0FEFFF5E7082194
:10536000307805F029FF6378002B00D047E72C4BFD
:105370002D4F0293E388029A04211380294B307841
:1053800003932389039A138063893B8005F034FEDD
:10539000002800D033E7264B1B68002B00D12EE7F6
:1053A000039902983A88098800881B68984726E77D
:1053B0004379132B00D022E70389012B0AD11D4B1F
:1053C0001B78022B06D10821307805F0F5FEFFF797
:1053D0002BFE14E7052000F095FD0821020030782F
:1053E00005F0D2FF0BE7C0462664FF1F051400003E
:1053F0002564FF1FC063FF1F9842FF1F7942FF1FF4
:10540000FA63FF1FDB63FF1FFC63FF1FFE63FF1FC9
:10541000CD63FF1F7042FF1FD463FF1FD663FF1FC2
:10542000CA63FF1FC863FF1FC663FF1FCC63FF1F54
:10543000BC63FF1FC463FF1F8020C001014200D076
:10544000E2E6CB0731D5324B1B78002B1DD0314E15
:1054500005AC3378052B1AD1023B23702E4B21006B
:105460001B7823722D4B1B7863722D4B187801F03B
:10547000DBFA002809D007202A4B30701B68002B6C
:1054800003D01B68002B00D098470120BCE60E20FB
:10549000254B06221B7825492370254B1B7863700A
:1054A00002ABC01805F068FED8E7022308001840D8
:1054B000194209D0174B1B78052B03D11D4B1888B7
:1054C00005F0BAFE02209FE60424214203D0FFF734
:1054D00037FD200098E6082308001840194200D143
:1054E00093E6154B1C78012C03D0022C0DD008201C
:1054F0008AE6124B124A134913481B8812880988FE
:1055000000880094FFF7E0FDF1E7FFF78DFDEEE77F
:10551000FE63FF1F2564FF1F7242FF1FD863FF1F3A
:105520002664FF1FC063FF1FDA63FF1F7342FF1F64
:10553000D963FF1F7042FF1FC463FF1F6842FF1F34
:105540006A42FF1F6C42FF1F6E42FF1F0200F0B550
:1055500001270A480A4E51188B1A002B00DCF0BDB7
:10556000082415784308684038404000805B013CBF
:1055700058406D08002CF5D10132EDE7FFFF000027
:105580007AB60011F0B500250F269D4200DBF0BD74
:105590004C5D070944403440A400A05801357840D0
:1055A000F3E70000F0B589B06A460D000B000F2745
:1055B000110010351C780133260024093E40167076
:1055C00054700232AB42F5D12023024AFFF7DAFFD2
:1055D00009B0F0BD80B60011F0B54E780B7889B0F7
:1055E00036020C00170001901E43012A61D9954B29
:1055F0009E4200D877E001339E421CD1062A17D183
:10560000CA788B7812021A430B791B0413434A7928
:1056100012061A438C4B5A6100221A705A808B4A28
:105620005A608B4A9A608B4ADA60002009B0F0BD5C
:1056300088225205EEE7884B9E423CD182498B7806
:10564000002B00D0F6E00C2A31D10F22A37893432F
:10565000E27812021343227912041343627912068C
:1056600013434B60E279A07912020243207A0004CE
:105670001043627A12060243CA60E27AA07A1202EA
:10568000024376484A81834208D804236E49142293
:1056900001980B7005F070FD1420C7E71201D218B5
:1056A00089235B059A42F0D801238B70BDE7022A5B
:1056B000FAD00523EAE76A4A01239642E6D1FFF7CA
:1056C000B3FC052F0CD9E378A2781B02134322798F
:1056D00012041A4363791B061343624A039313604F
:1056E00005F0F2FEA1E7584D2B78002B9DD1AB7849
:1056F000002B00D1A0E02B8901339BB20093B34271
:1057000000D091E0132AD4D9CF7C8B7C3F021221A8
:1057100020001F43FFF71AFF874200D08EE0002EC3
:105720003DD1E378A2781B0213432279E968120481
:105730001A4363791B06134303930A228B4212D147
:10574000FF23A370E370237163716B89002B09D170
:10575000E37B227C1B0212041343A27B13431B092D
:1057600001336B8100226B89002B8ED0002A67D118
:10577000686837013818000B6B6900030390984282
:1057800005D9686105F020FEEB780133EB7068689D
:105790001022A11C381805F0AFFC2E8145E76F8957
:1057A000009A7B1E9BB293423AD1E278A378120210
:1057B0001A43237905A81B04134362796C68120607
:1057C0001A43EB6800920392211D0C22049305F00A
:1057D000D3FC0120260004A940421036FFF7E2FE68
:1057E000013F012F17D1009A0B232861824200D07C
:1057F0004CE704221C49200005F07EFC042203A98A
:10580000686805F0A9FBE968039AFF23914200D17B
:105810003CE7F73B3AE73100FFF7C4FE1036DFE71D
:105820000923B742A4D831E7009BB34200D9FCE674
:1058300007232BE7022329E7032327E7062325E78E
:105840000A2323E7FFFE00009C42FF1F0000011116
:10585000FFFF00005048593601FF0000FFFF001114
:1058600002FF000034F00040A842FF1F10B5034CB7
:105870000B000122210000F06BFA10BD2D5A00111F
:105880000B8870B506000D000224162B11D92B00D1
:105890000322094900F05CFA041E0AD1074B2A884A
:1058A0001B88191C934200D9111C300089B200F0EA
:1058B000EFFA200070BDC046595A00113A64FF1F2C
:1058C00010B54A780400013A0B000220012A07D8DB
:1058D0000A78002A04D005222000024900F038FA94
:1058E00010BDC046875A00110A7810B50B0004009D
:1058F0000220002A04D007222000024900F028FAE2
:1059000010BDC046335B00110A7810B50B000400CF
:105910000220002A04D009222000024900F018FACF
:1059200010BDC046995B001110B5034C0B000B2253
:10593000210000F00DFA10BDC95B001110B5034C39
:105940000B000D22210000F003FA10BD3B5C00119A
:1059500010B5034C0B000F22210000F0F9F910BD27
:10596000955C00110A7810B50B0004000220002A93
:1059700004D011222000024900F0EAF910BDC0460F
:10598000A55C0011002310B51322190000F0E0F906
:1059900010BD000010B5034C0B001722210000F0D1
:1059A000D7F910BDF75C0011002310B519221900BA
:1059B00000F0CEF910BD000010B5034C0B001B2207
:1059C000210000F0C5F910BD315D0011F7B58489E3
:1059D0000D0006000121002C22D000238268D3563E
:1059E0001778002B1EDA0C2C1AD90C3CA4B2131910
:1059F00040880093230002F086FE431E9841013048
:105A00007B06DB0F6B703F23013C1F40A4B2287064
:105A1000AF70AC80002C07D0B3680133AB600021BD
:105A20000800FEBD0020EBE7AC60F8E70B780370E0
:105A30004B8843704B881B0A83700B79C37004201A
:105A400070470420022B06D10020537811781B02E6
:105A5000009A0B43138070470B8803700B881B0A56
:105A60004370022070470420009983420AD1537882
:105A700010781B0203430B80D37890781B020343FA
:105A800000204B807047F8B50D004B7801240021B1
:105A9000461C03702B788B4201D82000F8BD6B7830
:105AA000B01C4F1C012B10D1890069184B880222B1
:105AB00033704B88B9001B0A7370691805F014FB2A
:105AC00004360434A4B2F9B2E4E7122359436B1844
:105AD0005A88043132705B8810221B0A737069186F
:105AE00005F002FB12361234ECE770B5049D140089
:105AF0001E00052B01D8042070BD637812781B02AC
:105B000013432B80E378A2781B02134302226B809D
:105B10002A71211D681D063E05F0E6FAB2B22A81FF
:105B2000E92AE8D82800A11D0A3005F0DDFA002096
:105B3000E2E7002310B50A789A4201D8900010BD20
:105B40009A008A185488013304705488DBB2240AFE
:105B50004470948884709288120AC2700430EAE714
:105B600010B51100029C062B04D004201022142B27
:105B700001D010BD022222714B7808781B0203432A
:105B80002380CB7888781B02034363800431601D37
:105B900005F0AAFA0020ECE710B50C788B780431F8
:105BA0005C43E4B203702200013005F09DFA601CF2
:105BB00010BD0420022B06D10020537811781B025F
:105BC000009A0B431380704710B50C000A8802310D
:105BD00005F08AFA208810BD70B504000D00049805
:105BE0001100012B01D8042070BD167852781202E2
:105BF000324302800200F13255701470E125002C0E
:105C000000D10C35023B9AB24280AA42EBD8023155
:105C1000043005F069FA0020E6E704200099834289
:105C20000AD1537810781B0203430B80D378907805
:105C30001B02034300204B80704710B50C000A88FC
:105C4000023105F051FA208810BD000070B5012125
:105C50001E000420049C0E400B4218D1CB40DDB244
:105C60008D4214D90A49DBB2098899420FD3230027
:105C7000EE331D703300580011184978165C090284
:105C8000314301332152D9B28D42F4D8002070BD86
:105C9000B442FF1F10B50C000A88023105F024FA47
:105CA000208810BD10B50C788B7804315C43E4B2C9
:105CB00003702200013005F017FA601C10BD10B50A
:105CC00011000298032B01D8042010BD14785278DB
:105CD000043B120222430280CA788C7812022243CB
:105CE00042809AB28280EB2AEED80431063005F069
:105CF000FBF90020E9E710B50C000B8803700B8856
:105D00001B0A43704B8883704B881B0AC3708A88B8
:105D10000430063105F0E8F9A088043080B210BDE7
:105D20000420012B03D100201378009A13707047D0
:105D300010B50C000B8803700B881B0A43704A884F
:105D40000230043105F0D0F96088023080B210BD15
:105D5000F0B589B003931E4B029242000700D05A5F
:105D6000019102F020F81325061E2DD0029B01247C
:105D70000370019B002B04D0001903999847001968
:105D800084B26B461B7A5BB2002B0FDA102138000D
:105D900002F01CFB1925002813D130003219E1B2A2
:105DA00002F066FC051E0CD10C34A4B2042304AA34
:105DB000380005A993800696948101F0AFFD051E79
:105DC00002D0300005F080F9280009B0F0BDC046CF
:105DD0003864FF1F70B505000C0000280CD00020AF
:105DE000814209D010222000044905F07DF90120EC
:105DF0002B7823736B78637370BDC046C0B60011F7
:105E0000F0B506000D0017001C0085B002291BD05C
:105E10000020102907D1022B07D0102B03D115E049
:105E20000020102C08D005B0F0BD69463800FFF7FF
:105E3000D1FF2A0069460BE069463000FFF7CAFF30
:105E400022006946380004E0022BE9D12A0039001B
:105E5000300005F0D1FAE6E7031CF02800D9F02362
:105E6000032008499AB2013A0B80D3170340064930
:105E70009B189B100B80D30F04499B185B100B8061
:105E80007047C046B842FF1FB642FF1FB442FF1F13
:105E9000034B1B888B4202D3024B4000C152704718
:105EA000B842FF1F3864FF1F014B4000185A70476B
:105EB0003864FF1F1722014B1A8070473864FF1F98
:105EC00070B505000E2005F027FB041E13D0D0236B
:105ED000037000230622837007494570033005F0E4
:105EE00003F9064B2100DA8A62811B7E2373044B7F
:105EF000187805F0D9F970BD5464FF1F4464FF1F82
:105F00000843FF1F262803D8024B4000C05A7047A1
:105F10000148FCE7BA42FF1FFFFF000070B5060012
:105F20000C00094D1C220021280005F02DF8074B1C
:105F30001E70074B1C7005F02FF80123002801D0BC
:105F4000002312202B7070BD4464FF1F0843FF1F05
:105F50006564FF1F70B505000D4C0800E260A1608C
:105F600010220021656005F0A7F9012803D1102156
:105F7000A06802F058FD10220021280005F09CF9CD
:105F8000012803D11021606802F04DFD70BDC046AC
:105F90004464FF1F70B5041E05D1002903D00622FA
:105FA0000D4805F0A1F80D4B1D78012D11D1002CE5
:105FB00005D102221A7005F0C7F8280070BD002232
:105FC0001A70074B1B78FF2BF7D02000FFF778FFE4
:105FD000F3E70025F1E7C0465464FF1F4464FF1F48
:105FE0000843FF1F030010B5002801D1002010BD99
:105FF00000780B4A002803D15988D1821B79137687
:106000001378022BF2D10023984200D1033313708E
:10601000044B1B78FF2B01D0FFF752FF0120E6E76E
:106020004464FF1F0843FF1F002911D000280CD033
:106030004B79012803D140225242134303E03F220F
:106040001340032802D001204B7170474022F4E72F
:106050000800FAE770B5094D0100287800280BD038
:10606000074C0622200005F03FF821002878FFF7B2
:10607000DBFF200004F0F8FF70BDC0466464FF1F22
:106080003E64FF1F00290AD0012808D13F224B7926
:106090009343C02B03D0403B5A425341981C704756
:1060A00070B5174D06002B78FF2B15D00A2005F090
:1060B00033FA041E10D0D0230370C83B8370114BF9
:1060C00011491B784670C3700622043005F00CF8A5
:1060D0002100287805F0E8F80C4B1B78012B0DD136
:1060E0000B4B1B68002B03D09B68002B00D09847FC
:1060F000084B04211878084A05F0DEF970BDC04647
:106100000843FF1F6464FF1F3E64FF1F6064FF1F9E
:106110008C64FF1F9064FF1F60EA0000014B9868C9
:106120007047C0464464FF1F014BDB681868704726
:106130004464FF1F074B10B5DA681368013313601E
:10614000054B1878FF2803D08021C90105F004F918
:1061500010BDC0464464FF1F0843FF1FF7B50E0083
:1061600002F0C8F8051E1CD00E4B06621F78002FE7
:1061700000D10778AB791020019305F0CDF9041E0A
:106180000FD0D0230380C73B8370019BE91DC370F0
:106190000622043004F0A8FF21003800E66005F074
:1061A00083F8F7BD0643FF1F014B18787047C046C0
:1061B0006464FF1F054B002805D1054B1A78054B79
:1061C000002A00D1014B18007047C0465464FF1FDD
:1061D0006464FF1F3E64FF1F014B58687047C04650
:1061E0004464FF1F024B1868431E9841C0B27047B9
:1061F0006864FF1F421E03000120152A03D9FF3BDC
:106200005A425341D8B27047F0B51C0000230E002B
:1062100085B0039002920B70029A934201D3002042
:1062200019E0E55C5A1CD2B2002DF8D00298511941
:106230008142F4DC0233DFB2A35C18000193FFF764
:10624000D9FF002807D0013D019A0399EBB23370C2
:106250008A4202D1E01905B0F0BDDB19DBB2DBE701
:1062600010B50C0002F09EF803001220002B03D0A2
:106270002100588804F0E8FF10BD000070B50E4DF5
:1062800084006359002B15D0186A002801D005F04E
:10629000FBF82B59586A002801D005F0F5F82B5966
:1062A000986A002801D005F0EFF8285905F0ECF8BD
:1062B00000232B5170BDC0467464FF1F1C4B70B58A
:1062C00004000E00150099420AD11A4B1B68002BDE
:1062D00001D1122070BD1B68002BFAD09847F9E756
:1062E000154B994215D1134B1B68002B0AD01B6824
:1062F000002B07D09847002804D1104B1C70104B7E
:106300001D70E7E729002000FFF7AAFF0028E1D170
:10631000F3E7080001F0EEFF0028DAD0037803204D
:10632000A342D7D12900300004F08EFFD2E7C04647
:10633000FEFF00007064FF1FFFFF00006D64FF1F81
:106340006C64FF1FF7B50400808801F0D3FF0025BF
:10635000A84203D00578A08802F008F81C4E3378D4
:10636000002B1FD0AB421DD11A4B28001978FFF724
:1063700077FF002818D000233370A3790820A7786E
:10638000A688019305F0C8F8011E0DD0D023037034
:10639000CA3B8370019B477086808371280004F09C
:1063A00083FF01E0002DE8D1A0880B4B8200D35879
:1063B000002B01D0FFF762FF1721A088FFF768FDCF
:1063C000A08801F027FDA08801F0FEFDF7BDC046C2
:1063D0006D64FF1F6C64FF1F7464FF1FF0B587B00E
:1063E0001D000CAB1B88070001930DAB1B8814200C
:1063F00002930EAB1B88160003930FAB1B88009112
:10640000049310AB1B88059305F086F8041E1AD080
:10641000D0230370CB3B47708370C67006222900DF
:106420000430002D11D004F05FFE019B2100638138
:10643000029B0098A381039BE381049B2382059B1D
:10644000A37404F031FF07B0F0BD04F09DFDECE74C
:10645000F7B5009308AB1B8807000C200D00160051
:10646000019305F059F8041E13D0280001F042FFF3
:1064700000280FD00078D0232370C93BA370009B65
:1064800021002381019B6770A580E680638104F071
:106490000BFFF7BD014B1878EDE7C0460843FF1F1F
:1064A00013B5040064890389C2888188C078009488
:1064B000FFF7CEFF13BD000010B5044C2068002884
:1064C00003D004F0E1FF0023236010BD7864FF1FB8
:1064D000A122F0B5818892004A43384B384F1B689F
:1064E00004009B189D2292009B18827989B01A6043
:1064F0003B68002B5FD01D78324B1B68002B04D00B
:106500005B68002B01D00020984726000836310038
:10651000E079FFF7B7FD237DE0710200E078049396
:10652000638A29000393238A0293E3890193A38852
:1065300000933300FFF752FFE378002B0BD1E28981
:10654000A379A18802920196E279280000920122A3
:1065500001F0DAFEE0703B68002B20D0FFF7ACFFC3
:10656000194D287800281AD0184B1978FFF778FEB3
:10657000002814D02B78E67808200793A78804F029
:10658000CBFF011E09D0D0230370CA3B4670837035
:1065900087808671079804F087FE00232B701721EF
:1065A000A088FFF775FCA08801F034FCA08801F0FA
:1065B0000BFD09B0F0BD064B9DE7C0463409FF1F37
:1065C0007864FF1F8C64FF1F6D64FF1F6C64FF1FE6
:1065D0000843FF1FF8B5070008000E0001F08AFE0F
:1065E000041E18D02620FFF78DFC051E00D125784B
:1065F000062004F091FF041E0DD00021062204F0B5
:10660000C3FCD0232370C23B21006770A370A68017
:10661000E8B204F049FEF8BDF0B585B001930AABCD
:106620001B78070002930BAB1B7808000D0000924B
:10663000039301F05FFE061E22D0102004F06CFFD1
:10664000041E1DD01022002104F09EFC2620FFF71E
:1066500059FC002800D13078D0232370C13BA370AF
:10666000009B21002372019B67706372029BA580CF
:10667000A372039BC0B2E3720C9BE36004F014FEB0
:1066800005B0F0BDF7B50D00019001F033FE071E17
:1066900020D00E2004F040FF041E1BD02620FFF760
:1066A00031FC061E00D13E78D0232380C53B062254
:1066B000A370F91DE01C04F017FD019B2A00638103
:1066C0000123DD401A401D40210022736573F0B2A2
:1066D00004F0EAFDF7BD0000F0B585B002901000AF
:1066E0000D0017000A9E039301F004FE041E31D032
:1066F000029B002B2ED1039B02795B0724D512232A
:1067000013430422002E08D10B99002905D10C99BE
:10671000002902D10D9900291AD01A430D9B22712C
:10672000002B00D0C9E0002E00D1CFE0002D00D01A
:10673000CCE0606A002801D004F0A6FE1C213000E5
:1067400004F092FD606205E002239A430E33D7E71E
:1067500093432371654BBA00D458002C00D1AAE0B2
:10676000002E10D0236A002B03D11C2004F0F4FC6F
:1067700020625E4BBA00D358186A002803D01C224E
:10678000310004F0B1FC0C9B002B12D0574CBB0025
:106790001D596B6A002B03D1162004F0DDFC6862E2
:1067A000BB00E358586A002803D016220C9904F065
:1067B0009BFC0D9B002B11D04C4DBC006659B36A5D
:1067C000002B03D1142004F0C7FCB0622B59986A47
:1067D000002803D014220D9904F086FC380001F043
:1067E00089FD051E67D0414BBA00D358002B62D0FB
:1067F0001A6A3420002A00D11C389A6A002A01D073
:10680000143080B20B9A002A01D01C3080B25B6A2F
:10681000002B01D0163080B204F07EFE041E4AD058
:106820001822002104F0B0FB2620FFF76BFB01903B
:10683000002801D12B780193D0232370029B2000E4
:1068400063700A23294EA370039BBD00A371AB594B
:10685000A780196A1830002905D01C22A06004F016
:1068600043FC200034307359996A002907D0030093
:1068700014221433E060029304F036FC02980B9B60
:10688000002B08D003001C221C330B9920610293BB
:1068900004F02AFC02987359596A002903D0162281
:1068A000606104F021FC6B462100187904F0FCFCC7
:1068B0003800FFF7E3FC05B0F0BD10220D9B0D99E9
:1068C0001B69A018236204F00FFC2CE70B9B002B24
:1068D00000D13FE7012D00D03CE7606A002801D0DD
:1068E00004F0D2FD1C210B982AE7C0467464FF1FF8
:1068F00010B5044C2068002803D004F0C5FD002327
:10690000236010BD6864FF1F0B4B07B51A68002A8F
:1069100001D100200EBD6946531C012012780731B9
:10692000FFF772FC0028F4D0027801231000184011
:106930001A42EED0EEE7C0468464FF1FF0B51F4F49
:1069400001203B6887B0002B25D09B78059300F091
:10695000B3FB002821D00A20FFF7D4FA04000B2053
:10696000FFF7D0FA164B05001E78731E9E413B6858
:10697000F6B2191DD878FFF757FB3B682900DA7A81
:10698000043303929A79019302920090330020001D
:10699000059A04F039FB07B0F0BDFFF7B5FF0028FA
:1069A00005D00620FFF7AEFA04000720D8E708203C
:1069B000FFF7A8FA04000920D2E7C0466864FF1F69
:1069C0006464FF1F70B50A4E040033780D00FF2B7E
:1069D0000DD0042004F0A0FD011E08D0D0230370C8
:1069E000CE3B45708370C470307804F05DFC70BDA0
:1069F0001843FF1F70B5040006200D0004F08CFD45
:106A0000011E0AD0D0230370CD3B8370054B447028
:106A10001B688580187804F047FC002C01D0FFF734
:106A200067FF70BD6864FF1FF8B5264F06003B681E
:106A30000D001124002B05D10522234B1B78134296
:106A400002D112242000F8BD204A10241268002A26
:106A5000F8D01278002AF5D0DB0719D52B789A1ECA
:106A6000012A1AD80C2004F077FB13243860002880
:106A7000E8D000230A22437029000670023004F097
:106A800033FBFFF75BFF041E0AD0FFF731FFD9E7A6
:106A900000F012FB0028E1D1E4E7002BE2D0D0E7C0
:106AA0000B4B1B78032BCDD11D20FFF72BFA094B85
:106AB00018800028C6D0084B04211878074A04F033
:106AC000FBFCBFE76864FF1F6564FF1F8464FF1F52
:106AD0006464FF1F6264FF1F9064FF1F60EA000090
:106AE000F7B50193194B14001A78052306000F001F
:106AF00012201A4221D0012920D1154B1D68002DEA
:106B00001BD002201F2C18D8002C02D0019B002B78
:106B100013D0104B1F221E706E1C0021300004F099
:106B200033FA01992200300004F0DEFA310020002F
:106B30002C70002F06D004F0EFFBFEBD064B122098
:106B40001D68DCE704F010FBF7E7C0466564FF1F33
:106B50008464FF1F1843FF1F8064FF1FF8B50F4EAA
:106B600012243368002B17D01B780F3C834213D1BB
:106B700000250B4F0221387804F01EFB094B04213D
:106B800038781D8004F018FB074B28001D803368FF
:106B90005C7004F079FB04002000F8BD6864FF1FFE
:106BA0009064FF1F7C64FF1F6264FF1F70B50128A3
:106BB00023D11B4C2388002B03D01A4A1578002DB3
:106BC00007D0194B1B68002B02D01878FFF7C6FFBF
:106BD00070BD3B2B02D93C3B2380F9E7134E0221C9
:106BE000307804F0E9FAFA222388920002215A430D
:106BF000307804F0C9FB2580EAE70B4B1B68002BBB
:106C0000E6D00B4B1B785B07E2D5084B02211878C6
:106C100004F0D2FA0022024B1A80FFF769FED7E790
:106C20007C64FF1F6064FF1F6864FF1F9064FF1F88
:106C30006564FF1FF8B51E4D2868002803D004F0D6
:106C400023FC00232B601B4E3068002803D004F087
:106C50001BFC00233360184F05243B7818002040AC
:106C6000234221D0154800F02BFA3B78234213D061
:106C7000202004F071FA2860002813D0202200217F
:106C800004F082F9202004F067FA041E306005D079
:106C90002022002104F078F9002004E0286804F0A4
:106CA000F3FB2C601320F8BD00F00AFAF4E7C046AD
:106CB0008464FF1F8064FF1F6564FF1F0C43FF1F78
:106CC00010B50A4C23681A1E0ED0002808D10130D6
:106CD000587004F0D9FA002805D02368002B02D0A0
:106CE0000021FFF787FE0122100010BD6864FF1F1E
:106CF000F7B5274E050033680191181E21D05C7846
:106D0000244F012C30D1FFF7FFFD002825D02000B3
:106D1000FFF7F8F80400412814D91F4B0221187816
:106D20001E4A04F0C9FB1E4B3C3C1C800222336807
:106D30005A703B78002B14D128000199FFF75AFEB6
:106D40000120FEBDFA2292004243002AEED0124BEF
:106D50000221187804F018FBE8E7FFF7D3F80200E7
:106D6000F3E700233B70EBE73B78002BE8D10320EF
:106D700004F0D2FB011E08D0D0230370CC3B457039
:106D800083703368187804F08FFAFFF7B1FDD7E706
:106D90006864FF1F6064FF1F9064FF1F60EA0000CB
:106DA0007C64FF1F10B51749838802008B4220D0F6
:106DB00011D815498B4217D0144900205B1899B29D
:106DC000012907D8926811785A425341D8B2FFF787
:106DD000F9FD012010BD0E4A00209B1807229BB22E
:106DE0009A424041C0B2F5E783681878FFF768FF20
:106DF000F0E7836899785A78090218781143FFF709
:106E000077FFE7E70A20000006200000F8DFFFFF19
:106E1000AFDFFFFF014B18707047C0461943FF1FDB
:106E200010B5064C207001F041FA207804F0FCF90E
:106E30000521207800F062FD10BDC0469064FF1F60
:106E40000BB273B50D00002B00DBC4E0884B187843
:106E500004F072FB041E0ED00378912B0FD0A22BEE
:106E600000D1A1E0834B1878FF2852D0210004F014
:106E70001BFA00284DD180200002684076BD43787F
:106E80000F2B76D013D8052B70D00E2BEAD180882B
:106E9000794B98422BD8794B98421BD8784B984223
:106EA000E0D1A3681878591CFFF774F838E03E2B3E
:106EB000D8D18378032B74D06CD8012B6ED0022BE1
:106EC000D0D1704B1B68002B23D05B68002B20D0E7
:106ED00098471EE06C4BC0180C28C3D804F0B4F8D7
:106EE0001DC2C2150BC20B0B0B3223C23C00674BF9
:106EF000C0180728B6D8664B1B68002B09D01B6842
:106F0000002B06D0200098470AE0A3681878FFF706
:106F1000C7F8200004F060F9ADE7A068FFF762F859
:106F200000289FD0F5E7A3681B78002BF1D0554BC4
:106F30001B68002BEDD01B68002BEAD021005548C0
:106F40009847EDE74F4B1B68002BE2D01B68002BE6
:106F5000DFD021005048F3E7504B1B68002BD8D0FE
:106F60005B68002BD5D021004348E9E7FFF7EAF939
:106F7000CFE780884A4B984203D04A4B984200D0D2
:106F800070E7464B1B68002BC3D05B68002BC0D05A
:106F90002100D5E7153B012BBBD963E7FFF798FA32
:106FA000B7E7FFF77DFAB4E73F4B1B78042B07D117
:106FB00000236A4613800179408800F0C5FCA8E7E9
:106FC000364B1B68002BA4D05B68002BA1D00100BE
:106FD000364898479DE7012421420AD0294B1B6877
:106FE000002B04D05B68002B01D0002098470120C3
:106FF00043E78B070AD5264B1B68002B04D05B6840
:10700000002B01D020009847022036E704212800F9
:1070100008400D4200D131E7254E3388002B21D0A6
:10702000013B9BB23380002B1AD1FFF7DBF800281D
:107030000AD0204B1C70164B1B68002B04D05B68D9
:10704000002B01D020009847FFF7C6F8694601F0F1
:1070500001FD6846FEF7FEFF1D20FEF753FF30805E
:1070600004200AE7024B187804F0A6F8F8E7C046B7
:107070009064FF1F1943FF1F0E2000000120000035
:10708000091000008864FF1FFEDFFFFFAFDFFFFF76
:107090008C64FF1F0C2000000B2000007064FF1F99
:1070A0000D200000132000006564FF1FFFFF00009B
:1070B0006264FF1F6064FF1F10B501F09BF910BDF3
:1070C000014B18607047C0468C64FF1F0B8800207E
:1070D000162B01D817230420014A13807047C0469D
:1070E0003A64FF1F00207047074A0300118881425D
:1070F00007D091880020994202D1013080001018F9
:1071000070470020FAE7C0469864FF1FF0B58F78FB
:1071100006000D00C5B01E2F15D1FFF7E5FF051EB7
:1071200003D10024200045B0F0BD00223B00310017
:10713000C078009200F0B2FB0400A81C00F0D2FB63
:10714000FF23EB70EEE7264B062403931B78FF2BFF
:10715000E8D0182FE6D87B08224A013BDB000292D8
:107160009A589446002ADDD0029AD3185B68002B07
:10717000D8D00878002802D14B78012B02D1062400
:10718000122FCFD107AFAB88697800976446AA6801
:10719000A047041EC6D1AB78029A5B08013BDB0016
:1071A000D318390030005B689847041E0BD1AB78C8
:1071B000042BB6D0039A310010782200009700F01B
:1071C0006DFB0400AEE76A78002AABD1AA7805A966
:1071D0003B88087130000A704B80FEF747FBA0E740
:1071E0001C43FF1FD0B600111D4B37B50500984258
:1071F0000BD000290AD1FFF777FF002805D11948E5
:10720000FFF772FF002800D0058037BD01291AD191
:10721000FFF76AFF041EF8D001235B420380A378C6
:10722000FF2BF2D0FE2B07D00023E078142200932E
:1072300029001E3300F032FBA01C00F053FB012399
:107240005B426380E1E70229DFD1013901F0BEF83A
:107250000028DAD12800FFF747FF041EDFD1D4E76A
:10726000FEFF0000FFFF0000022210B5074B524254
:107270001A80074801325A809A80DA8000F07EFA3C
:10728000044801F025F8002010BDC0469864FF1F97
:107290000D710011E97100110388F7B50400002B8E
:1072A00002D102252800FEBD42680221137825483C
:1072B0005268FEF7A5FD00282ED0234F01253A88FD
:1072C000002AEFD0802321885B0201259B1A994276
:1072D000E8DC0C2003F040FF061E31D03B882288FA
:1072E0009C4600231800019561469DB2491989B258
:1072F000AA421BD8002801D062443A800023300003
:10730000082208C0210003F0EFFE104A1368002B8A
:1073100013D100251660C5E76268022113780C4876
:107320005268FEF76DFD0028C7D1BAE760681D01FD
:107330004019418101330198D6E71A001B68E6E73E
:107340001325AFE73EB700111A43FF1F9464FF1FD8
:107350003CB70011014B18707047C0461C43FF1F1B
:1073600014230A0010B51A40194204D0012210213A
:1073700001F048F810BD4B06F9D4012088434000C5
:10738000F8E710B514008B0604D50122102101F096
:1073900039F810BD08230A001A40194202D14BB235
:1073A000002B0FDA102101F02DF8002808D023005F
:1073B000F2331B78002BECD0F1342378012BE8D189
:1073C0000020E6E703208907FAD4E2E7F0B51F00C2
:1073D000184B85B01C68019002910392002C27D1B4
:1073E000200005B0F0BDA5683301ED186B89019A46
:1073F000934211D3029A93420ED8002F04D10A9BD4
:10740000002B10D12C00EBE73B002978039A686829
:10741000FEF7F6FC0028F2D10136B6B2A388B342DB
:10742000E1D82468DAE7A3680A9A5B891380E9E760
:107430000026F3E79464FF1F37B50C000A884988DB
:107440000123914217D3002A15D0651D23792A0004
:1074500002210A48FEF7D4FC102300280BD0237920
:107460006188208800242A000094FFF7AFFF0A23D8
:10747000A04200D0230018003EBDC0463EB7001118
:1074800013B50A0008884988012388420BD80028D0
:1074900009D00024137905320094FFF797FF0A23DF
:1074A000A04200D02300180016BD13B50A000888BA
:1074B0004988012388420BD8002809D00024137979
:1074C00005320094FFF782FF0A23A04200D0230078
:1074D000180016BDF0B58BB003904A8808880E00DE
:1074E0000123824255D3002853D00023012704AC46
:1074F00023700022718813000092FFF767FF051EBA
:107500003ED02078002835D12B78022B18D1677017
:107510006A8983000130E31880005A80696802227A
:10752000201803F0E1FD23780133DBB22370042B34
:1075300019D93B006889013080B2002BD9D01FE0F7
:1075400002236370122358436A89231804305A8037
:1075500069681022201803F0C7FD23780133DBB2DD
:107560002370002BE5D10C4A6B899B185A4253417A
:10757000DBB2DFE76378012BE4D12B78022BC7D095
:1075800022780A23002A04D021000398FEF798F9F4
:10759000002318000BB0F0BD0100FFFF0F4BF0B54A
:1075A00004001868002816D083685D89A54207D8B2
:1075B0008288AE18B44203DA12019A18934201D1BC
:1075C0000068EFE71E005F891036A74204D100294A
:1075D00000D00D801800F0BD3300EFE79464FF1F6A
:1075E00070B505000C0008880021FFF7D7FF0300E5
:1075F0000120002B04D022002800197AFFF7C1FED9
:1076000070BDF7B50C00002501902300EE331B7808
:10761000AB4201D800200AE06B00E65A002130009E
:10762000E718FFF7BBFF002802D126800130FEBD1E
:10763000017A0198FFF794FE002802D03B8823804E
:10764000F5E70135EDB2E0E710B504000888002148
:10765000FFF7A4FF03000120002B03D02000197ABC
:10766000FFF77EFE10BD0000054B1B68002B01D10B
:10767000180004E09A6852898242F6D198887047CF
:107680009464FF1FF0B50E27002687B0039302AB6A
:10769000FF183E8005001F4B40891400984207D018
:1076A0002B78013000976A6880B2FFF78FFE0600E2
:1076B00002212B7818486A68FEF7A2FB00280FD039
:1076C0006C892000FFF7D0FF002802D0013C04198C
:1076D000A4B2039B002B00D01C80300007B0F0BD8B
:1076E00002212B780D486A68FEF78AFB0028E7D153
:1076F00002212B780A486A68FEF782FB002807D02F
:10770000002EDED03B88A342DBD17489013CDFE749
:107710006C89DEE7FFFF00003EB700113CB70011A7
:107720003AB7001110B50C00FFF7DEFC0300022091
:10773000002B0AD0002C00D023609B781720FE2B52
:1077400003D00138FF2B00D1002010BD73B50D0010
:1077500001A904001600FFF7E5FF172805D0002E49
:1077600004D129002000FEF727F976BD012210215F
:10777000200000F047FE0028F3D0F6E7014B186028
:107780007047C046A464FF1F37B56B469D1D0100BE
:1077900004000222280003F0EFFC2B88B02B0ED14E
:1077A0002379122B09D12300FA331B78012B06D140
:1077B0000121608800F0E0F801E01B2BF8D037BD14
:1077C00010B5054B0421187000F098F8FFF74CFD38
:1077D000FEF770FB10BDC046A864FF1F0020F0B587
:1077E0000BB20F0087B0834234DA274B187803F0CE
:1077F000A3FE051E2BD00378A02B25D103AE3100AC
:10780000FEF7E4F8041E0BD1B378DB0724D51F4B39
:1078100006341B68002B03D03100688898470400A9
:10782000A868002801D003F04FFC002C08D1184AAA
:10783000039B1340174A934206D0B3781B2B03D007
:107840000121688800F098F8280003F0C5FC80202A
:107850000002784007B0F0BD0F4B1B68002B10D022
:10786000310068889847041EDAD07378002BD7D18E
:10787000B27801A90A704B800C716888FDF7F6FF99
:10788000CEE70624F1E7C046A864FF1FA064FF1FEF
:1078900000FFFF0000011200A464FF1FF7B5019074
:1078A000FC200D0017001E0003F036FE040013201C
:1078B000002C12D0B02320002370089BF4226770A4
:1078C000658026710830002B08D0190003F00CFCED
:1078D0002100019803F0E8FC0020FEBD089903F0A8
:1078E00053FBF5E710B5041E06D00078FD2803D839
:1078F00003F00AFCFF23237010BD00000A1F93B29F
:1079000010B504000220032B05D882400020024B52
:10791000D1529B189C7010BDC864FF1F0B8870B5B6
:10792000043B04000D000220032B0BD80121200092
:1079300000F04CFD03001420002B03D02900200090
:1079400000F0DEFB70BD000007B51300034A009293
:107950000A00012100F02CFC0EBDC046857B001101
:1079600007B5019203220092024B0A00122100F097
:1079700049FC0EBD037C001107B56B4601AA1180BE
:107980000449D88008780633012802D1190003F091
:10799000ABFD07BDA964FF1F0C4B10B51870002389
:1079A000FF210B4A1380138193819380094A5380EE
:1079B0001370517293819372D174D382137551777E
:1079C00003F06AFC00F0FCF910BDC046D864FF1F4C
:1079D000C864FF1FAA64FF1FF0B58DB06B4600207E
:1079E00003910C229B5E834200DBB0E05D4B187874
:1079F00003F0A2FD051E00D1A4E00378902B00D077
:107A00009DE006AF01004688380000F013FA79685F
:107A10000400002900D19CE03B88052B6ED13B89F6
:107A2000032B1CD905AC200000F0A2F86288172AAD
:107A300061D83989131D994231D17968237804318D
:107A40000291D90738D5607800F08EF9071E06D06C
:107A5000002303712378012B08D0132B23D0A868AF
:107A6000002800D178E003F02FFB75E062880299CE
:107A700009A800F0A6F80290380000F08BF909AAD6
:107A80002378387A0192002231000092029A00F0A5
:107A900012F9380000F064F9029B002BDFD03000AF
:107AA00000F080F9DBE70378032BD8D162880299D4
:107AB00009A800F0D6F8DEE7122B13D1029909A825
:107AC00000F0B5F8021EEAD127498B88002BC6D0FA
:107AD000887909A92378019161780091310000F03B
:107AE000EAF8BCE7002302AA93833000617809AA70
:107AF000FFF72AFFB3E71D4B0993F6E7042B02D0EB
:107B00009A1F012AABD8184A043B9B00995A0029B6
:107B1000A5D0D218907831003A0000F0AEF80028D5
:107B20009DD13B88042B03D001213000FFF724FFB7
:107B3000012C04D1A868002801D003F0C5FA280060
:107B400003F04AFB8020039B0002434018000DB065
:107B5000F0BD012800D182E701213000FFF70CFFC2
:107B6000EDE7C046D864FF1FC864FF1F010017007F
:107B70000B7803704B784370CB788A781B021343E1
:107B8000438070470A88030002700A88120A427014
:107B90000A88012A06D14A8882704A88120AC2706D
:107BA0000420704702208242FBD14A8804309A7038
:107BB0004A88120ADA708A881A718A88120A5A71F7
:107BC000EFE710B50400012082420CD94B780A7807
:107BD0001B0213432380834206D1CB788A781B0291
:107BE00013436380002010BD022BFBD1CB788A7831
:107BF0001B02134363804B790A791B021343A38052
:107C0000F0E70B8803700B881B0A43704B88837066
:107C10004B881B0AC3708B8803718B881B0A4371C6
:107C2000CB888371CB881B0AC3710820704703007F
:107C30000120082A14D14A780878120202431A80D7
:107C4000CA788878120202435A804A790879120267
:107C500002439A80CA798879120202430020DA80AE
:107C6000704710B504000120022A05D100204B788E
:107C70000A781B021343238010BDF8B506001020BC
:107C80000F00150003F048FC04000120002C0ED06A
:107C9000A0230C22290023806780201D002D07D0FF
:107CA00003F022FA2100300003F0FEFA0020F8BDB4
:107CB00003F06AF9F6E7F7B51E00009008AB142050
:107CC00017001D78019103F027FC041E12D0A22397
:107CD0000370019B47704380099B057146710C221C
:107CE0000830002B07D0190003F0FEF9210000989E
:107CF00003F0DAFAF7BD099903F046F9F6E737B56C
:107D0000041E0FD04388002B0CD00025C1881323FC
:107D1000007A172201950095FFF7CDFFFF236580BC
:107D20006372257037BD000010B50C4904004A8805
:107D3000002A09D08B89002B05D00020CB8A022293
:107D4000834201D010BD012213000A2043430020CA
:107D50004032C854C81842800472F3E7AA64FF1F77
:107D60000023438003707047094B00211A0010B5AF
:107D70005C88002C06D01C79844203D10A234B4333
:107D8000D01810BD01310A330329F1D10020F8E7E2
:107D9000AA64FF1F10B50400407A03F0B5F9FF2371
:107DA000637210BD7047043010B580B203F02CFB35
:107DB000002803D00421494203F0F6F810BD00006A
:107DC00070B50025104CA0682580A581A580A8422B
:107DD00002D003F079F9A56000250C4C0C4B606DC6
:107DE0001D80230058331D70A84202D003F06CF9A7
:107DF000656500256068002801D003F065F901354C
:107E000008340A2DF6D170BD7065FF1F1465FF1F81
:107E10006465FF1F70B5041E09D1054D2880A88137
:107E2000A880A868002802D003F04EF9AC6070BDAD
:107E30007065FF1FF0B54B8885B001930023436048
:107E40000A7905000F00022A00D07BE0CA88032AC5
:107E500017D98B685E7819783602DC78D8790E43AA
:107E600099781B7A24021B020C43034353495BBAE3
:107E70000B80331D93421ED1042C04D0631F022BB0
:107E80000ED9012015E0019A4D4B1201D35A002B57
:107E900006D00198FFF7BEFF4A4A13690133136108
:107EA0000421B8682E812C80494203F07DF8686077
:107EB000002005B0F0BD434D042C06D0631F022BFB
:107EC0000FD9EB680133EB60DBE7019A3C4B120101
:107ED000D35A002B05D00198FFF79CFF2B69013383
:107EE0002B61374B30000293019B029A1B010193D7
:107EF000002301998C468B52130063449C800393AA
:107F00009E81FFF750FF039B041E986016D004214A
:107F1000B868494203F048F8FA880100043A2000A2
:107F200003F0E2F80199029AFB888A5A043B9B18F5
:107F3000029A8B522B6801332B60A2E7AB690133A5
:107F4000AB619EE71E4B0293019B1E01029BF35AFD
:107F5000002B2DD002998C19A068002828D0012A66
:107F600026D1FA889B189BB27352A189994217D3E4
:107F70009B1AC018B96803F0B7F8029BA289F35A9C
:107F8000934200D07DE700222B81A3882B80A36839
:107F90006B60029BF2520B4A53680133536070E7E7
:107FA000084A9368013393600198FFF733FF68E74D
:107FB000044A536901335361F6E7C046DA64FF1F90
:107FC0007065FF1FE064FF1F70B5051E15D10B4CD7
:107FD0000B4B1880230058331870606D002802D0B6
:107FE00003F072F86565250050356068002801D0FF
:107FF00003F06AF80834AC42F7D170BD1465FF1F76
:108000006465FF1FF0B51700A12285B092000193AF
:108010004243394B06001B680C009B18D933FF33D1
:108020001D78FDF741FF0430854204DD3000FDF787
:108030003BFF0430C5B2BD4207D33A0000213000F7
:10804000019B03F0B1F905B0F0BD2900380003F041
:108050009BF82300C6B250331E700393019B290086
:108060006365380003F0F8F8CBB20293002B02D01E
:10807000039B01361E7000262300503303931B78A8
:10808000B34204D8606D002831D10020DBE7029AAA
:108090002800002A04D0013B1000B34200D0280081
:1080A000F700E719387003F017F9786000280ED050
:1080B0003A78019903F018F8019A3B780136D31801
:1080C0000E4A0193D369F6B20133D361D4E7039B1F
:1080D00018706065A74205D1084A1320D36A01339E
:1080E000D362B0E7606802F0EFFF0834F2E702F015
:1080F000EBFF00236365C8E73409FF1FE064FF1F3F
:10810000F7B50D0007000421686802F04DFF2B89C8
:10811000040003702B891B0A43702B8883702B8803
:108120001B0AC3702E8902250436F6B2F42E15D828
:108130001B4B9F4214D10C2003F0EEF91135011EA8
:108140000CD0902303708E3B0371043B4380154B8E
:108150008460C680187803F0A7F800252800FEBDCB
:108160005C237B43104AD3180093583301931B7848
:10817000002B0FD10300320038000099FFF742FFB7
:10818000019B05001B78002BE8D13800009903F013
:108190001BF8E3E7054A0725536A01335362DDE71D
:1081A000FEFF0000D864FF1F1465FF1FE064FF1F7F
:1081B000F0B587B0009017200F0016000193FFF76D
:1081C000F2FD1325041E19D00C98031E02D001994C
:1081D000201D9847030AE370052302AAA07004300B
:1081E000908127700098667003A993800494FFF72C
:1081F00087FF051E02D0200002F066FF280007B0AE
:10820000F0BD0000F0B587B01F000CAB1B780391E8
:10821000059301210DAB06001C78049200F0D6F8FE
:108220001425002821D02000FFF77EFD0135041E13
:108230001BD01149059B0A7803700132D2B2131E7C
:10824000C68001D101231A000B7022713000049BFB
:1082500003990097FFF7ACFF051E09D12300210009
:108260000648074A093302F0DFFE280007B0F0BDD8
:10827000002363802370F8E7DC64FF1FFF7C00119C
:1082800030750000F8B505000E00064C064F236857
:10829000002B02D03100280098470434BC42F6D1AC
:1082A000F8BDC0468065FF1F9465FF1F0123064A85
:1082B0005B425380002313715362044A136053607E
:1082C0009360D360136170479465FF1F8065FF1F43
:1082D0000200002310B506499C000859002801D16E
:1082E000625010BD0133052BF6D11320F9E7C046CB
:1082F0008065FF1F034A5388181A43425841404281
:10830000104070479465FF1FF0B585B002930AAB2B
:108310001F780CAB1B88009008000E00019203939D
:10832000FFF7E8FF05001120002D1BD10E48FFF7D5
:10833000E1FF04001520002C14D006220B99A77130
:10834000E01D02F0D1FE019B30002371029B290049
:108350006371009B66802370039B6562E381FFF776
:1083600091FF280005B0F0BDFFFF000010B5FFF73A
:10837000C1FF04000220002C12D060880121FFF709
:1083800081FF606A002801D003F07EF828220021D6
:10839000200002F0F9FD012300205B426380207180
:1083A00010BD000030B5074A074C5588010013780E
:1083B0000020A54204D05B1A59424B41584210405C
:1083C00030BDC0469465FF1FFFFF0000084A10B58E
:1083D00001230C00904208D0FFF78CFF031E04D04D
:1083E000037923405A1E9341DBB2180010BDC046EA
:1083F000FEFF0000024B1879431E9841C0B270473F
:108400009465FF1F70B504000D001600FFF772FFA2
:10841000002804D10D4B9C4200D0143070BD416A3D
:1084200003790520002907D012221A40102A02D110
:108430000520002EF2D10F20DB06EFD5897E0C201F
:10844000A9428941494249420840E7E7FEFF00004E
:10845000030010B5002800D110BD0348034A41882D
:108460009142F9D09847F7E79465FF1FFFFF00009E
:10847000002330B5C45CCD5C6C40D4540133102B68
:10848000F8D130BD0F23002210B5C45C6400224334
:10849000CA54C25CD209013BF7D210BD02000100F0
:1084A00010B52032103102F047FE10BDF0B58BB090
:1084B0000390102005931700049102F04DFE0090E8
:1084C000102002F049FE009B13240190002B05D0E0
:1084D00000280CD11324009802F0D6FF019B002B3A
:1084E00002D0180002F0D0FF20000BB0F0BD102029
:1084F00002F032FE0600102002F02EFE13240500CA
:10850000002E00D1AEE0002819D01022002102F088
:108510003BFD32002900039802F00EFE041E0ED12E
:1085200033787F2B51D830000099FFF7ABFF009BC9
:108530001B787F2B53D801990098FFF7A3FF3000D9
:1085400002F0A2FF002D02D0280002F09DFF002CB7
:10855000C1D1102002F000FE0600102002F0FCFD48
:108560000290002E7CD0002878D03A000F322300F1
:108570000125121105D00F333B4015B25A42534129
:108580001BB26A1E1201002B33D0049BD2B2981882
:108590000099029AFFF76CFF013D10220021300084
:1085A00002F0F2FCADB2049F2D017D19AF4242D022
:1085B000002C33D0300002F067FF029B002B00D16B
:1085C00089E7180002F060FF85E729003000FFF717
:1085D00059FF28002549009AFFF74AFFA7E729001D
:1085E0000098FFF74FFF28002049019AFFF740FF4E
:1085F000A5E70F210F4004998A18D9B28F4208D9F4
:10860000D15C06A819540133102BF6D1029A0199B6
:10861000C0E7791A48424141C901F2E73900300008
:1086200006AAFFF725FF3200039806A902F084FD91
:1086300010370400BAE7002CBCD13000029906AA1A
:10864000FFF716FF320006A9039802F075FD082215
:1086500004003100059802F047FDABE71324A9E7B9
:108660001324AAE7002800D06EE733E744B70011CF
:10867000F0B58BB00F0016000225009000283FD007
:10868000002A3DD00B1DDBB21800029302F064FDFE
:108690001135041E34D0FDF747FD05003A0000995E
:1086A000201D02F021FEEBB20393E3702B0CDBB232
:1086B0002F0A00936370FFB22B0E2370A7700193F3
:1086C000FDF72CFD1022010006A802F00DFE21008E
:1086D000029A04AB06A8FFF7E9FE051E0DD1039B25
:1086E00008223370009B04A9B370019B7770F3706C
:1086F000301D02F0F9FDFDF71DFD200002F0C4FE63
:1087000028000BB0F0BDF0B58FB00D00149E0390A3
:1087100004920593002A03D1022420000FB0F0BD7B
:10872000002EF9D00398FFF7E5FD1424071EF4D0BE
:108730007278337812021A43B3781B041343F27829
:1087400012061A43036A0192934201D30133E3D123
:10875000002D03D03B7901249B07DED508220021A0
:1087600006A802F011FC059B13240433DBB21800A9
:10877000029302F0F1FC051ECFD0059A0499043053
:1087800002F0B2FD04223100280002F0ADFD3900F4
:10879000102210310AA802F0A7FD2900029A06ABA8
:1087A0000AA8FFF783FE041E0FD1082206A908A815
:1087B00002F09AFD0822311D08A802F01DFE0128D2
:1087C00007D101990398FDF7C9FC280002F05CFE6F
:1087D000A3E70124F9E7000070B51C4C05002368ED
:1087E000181E10D0002D14D11A78002A0CD1981C14
:1087F000083202F079FC02F0BFFE0135002808D1F2
:1088000023681D70012070BD0A331800082202F091
:108810006BFC2368002BF5D0122002F07DFE061EB3
:108820000DD0C1232168037045700231102202303F
:1088300002F05AFC23683100587802F035FD2068B8
:1088400002F022FE00232360DCE7C046BC65FF1F68
:10885000F8B504002020FDF755FB0D4EA700BB59CD
:108860000500002B0DD000280BD0D878FF2809D1A7
:1088700008492A000C55F35907480333611802F0E0
:10888000D3FBF8BD290002F05FFD0028F0D1F8E726
:10889000D865FF1FC065FF1FA99A001170B5064D6E
:1088A00084006359002B05D0D87802F02DFCFF22FC
:1088B0006359DA7070BDC046D865FF1F70B50600F9
:1088C0008CB00C00150000213022684602F05CFBE1
:1088D00031001022684602F007FD1D20210003220E
:1088E000684402F001FD6846FFF7D8FD2D21040021
:1088F00003222800694402F0F7FC20000CB070BD90
:10890000F0B50700160097B001931CAB1D7830221C
:108910001EAB00910AA800211C7802F035FB102242
:1089200039000AA802F0E0FC1022002102A802F09F
:108930002BFB0722310002A802F0D6FC072202AB73
:108940009818631E9C41019902F0CEFC02AB9C7307
:108950002B005A1E934102AAD3730021102206A8AD
:1089600002F012FB06221D9907A802F0BDFC1A2096
:1089700002ABC01806221F9902F0B6FC1022009923
:108980000EA802F0B1FC102202AB0EA908781C78E8
:10899000013A6040D2B2087001330131002AF5D1AA
:1089A0000AA8FFF77BFD102212A904000EA802F00E
:1089B0009BFB102206AB0EA908781D78013A68408F
:1089C000D2B2087001330131002AF5D10AA8FFF7AD
:1089D00065FD044310222098E4B212A902F084FC41
:1089E000200017B0F0BD70B50E0014008CB001006F
:1089F000102268461D0002F077FC3100082204A80E
:108A000002F072FC2100082206A802F06DFC684604
:108A1000FFF744FD04001022280008A902F064FCBE
:108A200020000CB070BDF8B506000D000024371909
:108A3000AC4200D3F8BD02F0B7FB030A3B70631CE5
:108A4000DBB201379D4203D90234F054E4B2EEE7C1
:108A50001C00EDE773B506000C000225002819D0B4
:108A6000002917D0032101A8FFF7DDFF6B469A7993
:108A70003F231A40013313436A463000937101A922
:108A80002200FFF71BFF051E04D10322E01C01A9F1
:108A900002F02AFB280076BD03785807DA08C00FD9
:108AA000D20080009B0710439B0F1843C0B2704751
:108AB00007230B40C908C9000B430370704700002F
:108AC00070B50400FFF7EAFE134DA4006359002BB4
:108AD00021D0186A002801D002F0D6FC2B59986EDC
:108AE000002801D002F0D0FC2B59D86E002801D00C
:108AF00002F0CAFC2B59186F002801D002F0C4FC08
:108B00002B59586F002801D002F0BEFC285902F002
:108B1000BBFC00232B5170BDD865FF1F0E4B80009E
:108B2000C35870B50C00002B0FD09D68002D0CD0E1
:108B30002B78201D0B706B784B70A97CFFF7B8FF6A
:108B40002B7E23726B69E36070BD10220021200030
:108B500002F01AFAF8E7C046D865FF1F014B18600B
:108B60007047C046D465FF1F074A03008000825843
:108B700010B5002A06D0D088984203D1012901D12E
:108B8000FFF79EFF10BDC046D865FF1FF0B5264E0B
:108B900095B087000B93BB590500099112200A92EA
:108BA000002B31D0D888FFF7A5FB04001420002C3F
:108BB0002AD0280010A9FFF7B1FFBB591E781D6A03
:108BC000002E23D00895FDF7EFFA07000020FDF7EF
:108BD000F1FA0790A379E61D069310AD0CA9089849
:108BE00000F0E2FA0EA9280000F0D7FA0B9B0A99D0
:108BF0000493069B09980293079B039601930097A1
:108C00000EAB0CAAFFF77CFE15B0F0BDFDF7CCFA59
:108C100006903000FDF7CEFAE31DA779079310AB5D
:108C200006000893DAE7C046D865FF1F30B50C4C44
:108C300085002A59030085B00120002A0ED01800B3
:108C40006946FFF76BFF2B591A78D888054B002A25
:108C500000D1054B6A46072100F0D9FB05B030BDB5
:108C6000D865FF1F9B910011A991001130B5094CE7
:108C70008500295985B010226846253102F034FA62
:108C80002A591121044BD0886A4600F0C0FB05B078
:108C900030BDC046D865FF1F4592001130B5094C64
:108CA0008500295985B010226846353102F01CFA3A
:108CB0002A591121044BD0886A4600F0A8FB05B060
:108CC00030BDC046D865FF1F83920011F7B54D4FE8
:108CD00086001020F4590D0002F03EFAF35920628C
:108CE000186A132200286CD0033A29009C6802F00D
:108CF000FBF9F3591A780192002A58D11E6A227D95
:108D0000317B944651400122019F114201D16746B7
:108D10001740217D914339432175377B4F40BC4635
:108D200060460027800701D44F0817400121022028
:108D30008F40227D82433A432275377B5740BC46A1
:108D400060460027400701D497080F400420227D89
:108D5000BF0082433A432275627D002794466046F5
:108D6000727B42400A4201D167460F400121627D79
:108D70008A433A436275777B5740BC46604600277A
:108D8000800701D457080F400220627D7F00824394
:108D900017436775767B00227E40760701D4BA08B8
:108DA0000A400426617D9200B1430A4362756A78E5
:108DB000002A08D06278002A05D005220533DA7728
:108DC00000221000FEBD04222979114205D1A17CA8
:108DD000114202D10533033AF1E7019A21782C7848
:108DE000002A02D10A002100140018220429E8D820
:108DF000042CE6D805206043034A05331218525C60
:108E0000DDE7C046D865FF1F54B7001110B50A0052
:108E10001121024B00F0FBFA10BDC046DF92001199
:108E20000B0030B587B001AD2B806B4604001100FC
:108E3000981D082202F058F92A000B212000024B4D
:108E400000F0E5FA07B030BD0793001110B50A0035
:108E50001121024B00F0DBFA10BDC0465B930011FC
:108E600013B50B0011006A4613706B46040006220E
:108E7000581C02F039F96A4608212000014B00F025
:108E8000C6FA13BD7B93001110B50A001121024BE5
:108E900000F0BDFA10BDC046CB9300117FB50500B0
:108EA0000B4BAA00D4580800002C0FD0666F237F0C
:108EB000E28821780396266F0296E66E0196A46EEC
:108EC0000094FDF709FC2800FFF7FAFD7FBDC046BE
:108ED000D865FF1F10B51721FFF7E0FF10BD000098
:108EE00070B50A000D00064B0221040000F08FFA55
:108EF000060029782000FFF7D1FF300070BDC04682
:108F0000AB92001170B586B000236A461370836877
:108F100004001D78681E0A2859D801A902F02CF80F
:108F2000060633373B3F43474B4F5300180000F0D2
:108F300042F9062312284BD000281BD16088FFF786
:108F4000D9F90823002813D04279002A47D1264BAB
:108F50001A78072312070BD5244B1A680723002A17
:108F600006D01668002E03D0290001AAB0470300DE
:108F70006A4613706B461B786088002B2AD1FFF776
:108F800067FC06B070BD180000F06CF9D4E718005B
:108F900000F087F9D0E7180000F093F9CCE718004B
:108FA00000F0ADF9C8E7180000F0C3F9C4E71800F5
:108FB00000F0F6F9C0E7180000F0F6F9BCE7180079
:108FC00000F013FAB8E7180000F013FAB4E707232B
:108FD0006A46137069466088FFF782FFD1E7052370
:108FE000012AC5D1024BB8E76564FF1FD065FF1F9A
:108FF000D465FF1FF8B52C4F8600F35904000D000F
:10900000002B40D0DA8882423DD15A78062A33D1EB
:109010001A78002A2ED0012099681A6A097D014227
:1090200006D0157B054203D007225A700120F8BDF7
:109030000220014204D0157B054201D00922F4E749
:109040000420014204D0127B024201D00B22ECE743
:10905000164B1B68002BE9D05B68002BE6D0200084
:109060009847BB5900215B78122BDFD12000FFF716
:1090700015FFDBE70E4BECE7112A04D1002900D0E5
:1090800032252900F2E7002D08D12000FFF732F940
:10909000002803D010230279134303712100280014
:1090A000FDF798FAC2E7C046D865FF1FD065FF1FDD
:1090B000D465FF1F70B50E4E8500AB590400002B20
:1090C00013D01B78002B11D10A4B1B68002B04D046
:1090D0005B68002B01D02000984773595B78122BF6
:1090E00003D100212000FFF7D9FE70BD024BECE751
:1090F000D865FF1FD465FF1FD065FF1F094B800097
:10910000C3581020002B0CD01A6A002A09D09B6883
:10911000002B06D0127A1B7E101C9A4200D9181C14
:10912000C0B27047D865FF1F70B503000D00140072
:109130000220002A30D000292ED013700B78081D91
:1091400053704B789370FFF7A7FCE0700120022169
:109150002B7A23716B7B034063716A7B0A40134354
:10916000042263716E7B1640334363716E7BF60895
:10917000F600334363712B7B0340A371287B0140CE
:1091800000200B43A371297B0A401343A3712A7B60
:10919000D208D2001343A37170BD10B50A000100BC
:1091A0000120FFF7C1FF10BD10B50A000100022029
:1091B000FFF7BAFF10BD70B506000C000220002EAC
:1091C00030D000292ED07378201D0B70B3784B70EF
:1091D000F178FFF76DFC01223579257271794B101A
:1091E0000800134093401040034388101040800053
:1091F000C9080343C9000B436373B1794B100800DE
:109200001340934010400343881002409200C90865
:109210001343C9000B4321202373FCF773FE8542DF
:1092200001D2122070BD2220257AFCF76BFE854208
:10923000F7D823781820042BF4D86378012BF1D8C1
:109240000020EFE7030010B50220002909D0002B11
:1092500007D00322481C0A7019000D3201F044FFA8
:10926000002010BD03000222080010B5002B06D01C
:10927000002904D00E32591C01F036FF00221000E4
:1092800010BD030010B50220002909D0002B07D023
:109290000422481C0A7019000C3201F025FF00203E
:1092A00010BD10B5FFF7DEFF10BD0300022000293E
:1092B00006D0002B04D0052200200A701B784B70CA
:1092C000704703000220002B08D0002906D05B78ED
:1092D00000200B70013B082B00D9183070470300A9
:1092E00010B50220002909D0002B07D00622481C07
:1092F0000A7019000A3201F0F7FE002010BD10B507
:10930000FFF7B0FF10BD02000B00022010B50029CE
:109310000ED0002A0CD007211970118859701188BD
:10932000090A997011180822D81C01F0DDFE0020EE
:1093300010BD03000A00022010B5002B0CD000293C
:109340000AD099785878090201431180901CD91CE1
:10935000082201F0C9FE002010BD030010B5022054
:10936000002909D0002B07D00822481C0A701900D8
:10937000921801F0B9FE002010BD02000B0002207F
:1093800010B500290BD0002A09D0092119701178D5
:1093900018185970511C062201F0A6FE002010BDBD
:1093A00010B5FFF75FFF10BD02000B00022010B5E3
:1093B000002A09D0002907D0517819701118062207
:1093C000581C01F091FE002010BD030010B50220D2
:1093D000002909D0002B07D00A22481C0A70190066
:1093E000063201F081FE002010BD10B5FFF73AFFF4
:1093F00010BD02000B00022010B5002A06D0002983
:1094000004D018005178FFF753FB002010BDF0B5D1
:1094100085B017001E006A460623050008009181EA
:109420009380FEF7C0FC1324011E02900CD038007C
:10943000B047041E05D1280001A9FEF76FFA041EEB
:1094400002D0029801F040FE2800FFF701FA200048
:1094500005B0F0BDF0B504008BB0019115000021FE
:10946000102202A801F090FD334EA700B859002841
:109470003CD0C388A34239D10378002B36D142783F
:10948000062A18D102000100553235310C3006ABE6
:10949000FFF7A9FA002829D12000FFF72FFE0200CC
:1094A00006A902A801F020FE200002A901F0CCFFCD
:1094B00001200BB0F0BD816E002917D00B8A112A54
:1094C00028D19D420ED101981231093A01F094FF42
:1094D000012807D1BB5920009D6EFFF70FFE290020
:1094E0000200DEE732212000FFF7D8FC2000FEF763
:1094F00001FF061E1BD0416A002918D00B8AAB421F
:1095000015D108220198123101F076FF01280ED101
:10951000716A0AE09D42E9D108220198123101F0F6
:109520006BFF0128E2D1BB59996E8A7EB9E7200012
:1095300001F032FFBCE7C046D865FF1FF0B56B4DA8
:1095400087007E5985B0337802900393002B00D0BA
:1095500087E0B368346A01937078062817D1012236
:109560001B7D134202D0217B114218D102221342EB
:1095700002D0217B114251D10422134203D0237B1C
:10958000134200D08BE0019B5A7DEB5991E00738E4
:109590000428F8D801F0F0FC032E42678300B36E74
:1095A000002B03D11C2001F0D7FDB066EB599C6E57
:1095B000002C1CD010220021200001F0E5FC0298B4
:1095C000FFF79CFD01002000FFF72DFA01F0ECFDF4
:1095D0002082200008211230FFF725FA0298FFF7B9
:1095E0008DFDA076EB592100D888FFF70FFC0822EB
:1095F000EB591CE0B36E002B05D01A00198AF088D5
:109600001232FFF70DFC0222019B197DEB5911422A
:109610003DD0207B10423AD0073208E0F488FCF7B6
:10962000DBFD01002000FFF711FC0A22EB595A7004
:10963000029B9C002A595378073B042B11D8D088F1
:10964000FEF758FE00284ED0C3895A08D218284980
:10965000029B0298CB542B5941180433254801F042
:10966000E3FC05B0F0BDFCF79FFD03000120834241
:1096700001D100200393EB59DE88FCF79BFD039991
:1096800002003000FFF7ECFB019AEB59117D042238
:1096900011420CD0217B114209D00B22C7E7F6887A
:1096A000FCF73CFD01003000FFF7EEFB6BE7019A91
:1096B000527D01210A4204D0607B084201D00C2275
:1096C000B5E702210A4204D0607B084201D00E2295
:1096D000ADE704210A4204D0627B0A4201D0102285
:1096E000A5E71222A3E7FA225200B0E7D865FF1FD0
:1096F000DC65FF1FB39A001110B5064B1A780423DE
:10970000100018401A4200D00348FFF727FA002043
:1097100010BDC0466564FF1F2043FF1F70B50400E5
:10972000FFF7D4FA051E43D12000FFF77FFA234E3E
:10973000A400A0598268937CDB0708D50321036A43
:109740001B790B40012B02D1017F0B430377431D93
:10975000D97F8B1E022B0DD8022900D00121C08891
:10976000FCF790FF042133591A7F59700A431A7786
:10977000280070BD01290CD1022310224370002162
:109780000C3001F001FC305910213530FFF74BF956
:10979000EEE70529ECD10223D118437010220C30DA
:1097A00001F0A2FC04233259117F0B431377EAE73F
:1097B00008251828DCD1053DDAE7C046D865FF1F2B
:1097C000F0B58BB0059143887E4F9E00F45915008B
:1097D0000493002C15D1012902D000200BB0F0BD5C
:1097E000101D57781678FFF757F9EB68320002938F
:1097F0002B7A0499019300903B002000FCF70CFFAA
:10980000EBE7E388049A934201D00820E6E7237847
:10981000012B00D1D4E0059B581E092800D9CFE0C8
:1098200001F0AAFB05CE0A29CC506C859AB229001A
:109830000498FFF773FFD1E720002900102245307C
:1098400001F052FCB9594B78042B02D1013B4B700B
:10985000C3E70B000A00253335320C310498FFF7BB
:1098600095F90498FFF702FA0522431E9841BB5967
:10987000C0005A70B2E7200029001022553001F0D4
:1098800033FC049B4F4C9D00295904980A0006ABF9
:1098900055320C31FFF77AF929591022453106A8C3
:1098A00001F0AAFD012808D10498FFF7F7F9059007
:1098B000002804D106222B595A7005988EE70823F8
:1098C0000593FAE763780C2B7AD1E36E002B03D172
:1098D0001C2001F041FCE066BB59D86E00286FD017
:1098E0001022290001F000FCBB590498DC6EFFF740
:1098F00005FC0D22A076BB595A706EE7E06E002879
:109900005ED063780D2B5BD12B8808220382A91CC3
:10991000123001F0E9FBBB599A68517D02221142D5
:1099200026D0186A407B104222D00C32E4E76378DC
:109930000E2B45D1236F002B03D1162001F00CFC18
:109940002067BB59186F002803D01022290001F0AE
:10995000CBFB0F22BB59CFE763780F2B30D1206FA1
:109960000622691C103001F0BFFBBB599A68517D7B
:109970000422114203D0196A497B1142D5D100213A
:109980000498FFF78BFA28E7636F002B0DD0BB59C3
:10999000586F0028F3D01022290001F0A5FB012206
:1099A000BB5952425B6F1A61E9E7142001F0D4FB06
:1099B000BB5960675B6F002BE9D126E72978DFE7A9
:1099C00007200BE7D865FF1F10B5064C207001F08B
:1099D000CBFA06212078FDF791FF0348FEF778FCCB
:1099E00010BDC046EB65FF1F698B001100200BB254
:1099F00070B50D00834216DA264B187801F09CFDF5
:109A0000041E0DD00378922B0ED0A02B37D0224B02
:109A10001878FF283AD0210001F046FC002835D103
:109A200080200002684070BD43780E2B0BD03E2B87
:109A3000EDD18378052B12D0082BE8D1817980886D
:109A4000FFF7D8FA08E0154B82889A42DFD1836885
:109A50001878591CFEF7C0FE002817D1D7E7104B25
:109A60001B785B0712D50F4B1B68002B0ED09B6831
:109A7000002B0BD0C289811D80889847ECE7FFF747
:109A800041FAA068002801D001F01EFB200001F07F
:109A9000A3FBC5E7EB65FF1F1943FF1F182000005C
:109AA0006564FF1FD465FF1F10B50078FFF712FA39
:109AB00010BD10B50078FFF7FDFA10BD0C2343432D
:109AC000084A10B59B185A68002A03D0012901D111
:109AD000904710BD9B68002BFBD00029F9D1984717
:109AE000F7E7C0460866FF1F01238340094A10B507
:109AF000946B1C439463506B98435063D46B200069
:109B00009843012901D120001843D063116B0B4306
:109B1000136310BD00800040F0B500240127154BF1
:109B200085B0DA6B144E03921A6C0192DA64019BD1
:109B3000E3403B4217D0039DE5403D400295E5B22E
:109B400002992800FFF7BAFF316A736A002908D02A
:109B50003900002B01D0029979402800FFF7C4FF9B
:109B600001E0002BF9D101340C36172CDFD105B000
:109B7000F0BDC04600800040EC65FF1F064B012190
:109B80005A68C2400A4204D01B68C340180008400B
:109B900070471B6DF9E7C0460080004030B50324D4
:109BA00044430F4BE25C1B199C785D7801232D1B0D
:109BB0000135AB40013BA340A140DB430C00122820
:109BC00007D80849920052181168194021431160C2
:109BD00030BD054A11680B4023431360F8E7C046C7
:109BE0009BB7001108F0004014F00040C21F70B590
:109BF000D4B20623092C0BD80125084C9540002926
:109C000008D00021FFF7CAFF23682B4323600023FD
:109C1000180070BD2368AB43F8E7C0460038004029
:109C2000214BF0B51B185B78022B21D10324444350
:109C30001E4A1F4EA35C121994780122150085401C
:109C4000B76B013CE4B23D43A240B563194C122806
:109C500015D89B0000290CD117495B1899680A4355
:109C60009A600123205C154A834011680B431360FE
:109C7000F0BD11495B18996891439960F1E70E4B6B
:109C800000290DD159690A435A61225C1328E8D092
:109C90000123203A93400A49086803430B60E7E731
:109CA000596991435961F0E7EC65FF1F9BB70011BB
:109CB00000800040E0B7001100F00040A0F000403C
:109CC000A4F00040F8B500241B4E1C4D1C4B1B5D3E
:109CD000012B1FD1194A9269E2401A420BD001228E
:109CE000B25693402200143AD2B2022A09D815493A
:109CF0004A6913434B61013402360C35172CE5D108
:109D0000F8BD0022B2560F499200521891680B43D9
:109D10009360F0E7022BEED1E7B23800FFF72EFF99
:109D200001235840C1B23800FFF77AFF3800FFF72F
:109D300025FF6877DFE7C0466DB70011EC65FF1FB0
:109D4000ED65FF1F00F00040012202388240054B04
:109D5000002903D059690A435A61704759699143F0
:109D60005961FAE700380040F8B50E0001210F00F4
:109D70008740114A0400D368FD43BB43D360831E70
:109D80008B4201D8FFF7E0FF00212000FFF72EFFF4
:109D90000A4A0B4B5168012E05D139431B195160FA
:109DA0005E700020F8BD2940516002221C196270CB
:109DB0009A6915409D61F4E700380040008000403A
:109DC000EC65FF1F012210B58240074B002906D029
:109DD00019680A431A600121FFF7C6FF10BD196810
:109DE00091431960F7E7C046008000400C2370B52E
:109DF000002543430A4A29009B181D70094B0400A3
:109E00001B185D70FFF7B0FF0123A340064928002F
:109E10000A681A430A6005490A689A430A6070BDD5
:109E20000866FF1FEC65FF1F348000403080004053
:109E3000F8B50C244443134B0500E4186368002B69
:109E400003D1A3681220002B1AD0022201270E4B47
:109E500000215B195A7028002770FFF785FF63689F
:109E60001E1E08D0A3683E00002B04D02800FFF778
:109E700085FE4640F6B228003100FFF735FE00208F
:109E8000F8BDC0460866FF1FEC65FF1FF7B5C4208C
:109E9000FF222B4B80001958002491433F3A0A437C
:109EA0001A508022274F5202274E1A60274B1D5D01
:109EB000002D21D0A31E012B03D80121E0B2FFF712
:109EC00043FF012D18D11F4B9B69E3402B4213D058
:109ED000E3B218000193FFF751FE01000198FFF76C
:109EE00071FFE3B2143B022B1DD801217156184AB1
:109EF0008D405369AB4353613B7F002B0DD0E5B2DE
:109F00002800FFF795FF2800FFF738FE7B7F010050
:109F1000834202D02800FFF7D1FD01340C3702360E
:109F2000172CC3D1F7BD012100237156F3568D4084
:109F3000074A9B009B189A68AA439A60DCE7C046D0
:109F400000E100E0EC65FF1F6DB70011ED65FF1F3C
:109F500000F0004010B501210400FFF705FF0123C8
:109F6000044A002011194B70A34091690B4393617F
:109F700010BDC046EC65FF1F70B50E001500040053
:109F8000FFF734FF0C236343094A20009B189D60B0
:109F90005E60FFF74DFFF021064B074A8900051E62
:109FA0005A5002D02000FFF721FF280070BDC046A4
:109FB0000866FF1F0000FF1F199B001170B5134DAD
:109FC00007202C78002C1FD1982221005200280055
:109FD00001F06AFA0123C420FF222B700C4B800091
:109FE0001C635C630B4B1C605C600B4B195891430A
:109FF0003F3A0A431A50802252021A600D20074A43
:10A00000074901F009F9200070BDC046EC65FF1F4B
:10A0100000800040A0F0004000E100E08D9E0011B3
:10A02000C59C0011030010B50620072B09D8054A6E
:10A03000137000F0D1FFD7210020034B034A8900A1
:10A040005A5010BD4843FF1F0000FF1F8D1BFF1F0C
:10A0500070B51D0002240C2910D8094ACA40D20745
:10A060000CD5FBF75BFF041E08D1059A0499280064
:10A07000FBF770FFFCF7DEFDFFF73EFB200070BD35
:10A080001210000030B50D7802232C009C431842BA
:10A0900001D02B431C0008252300AB43284201D0EC
:10A0A0002B00234320241D00A543204201D01C4344
:10A0B00025002A230D70184204D011781E3B0B4353
:10A0C000137030BD0028FCD10C2113788B43F7E7C7
:10A0D000F8B51D0006AB1B88140007AA0E000B2064
:10A0E0001778002B27D10A78022A49D14A6850787C
:10A0F00011780002244A08438018042840D800F050
:10A100003BFF03121D1B2300F06800F0B5FF021C8B
:10A11000C0B2B84200D93A1CD2B22000F1682A80FD
:10A1200000F0E2FF06E00222F3681B882A80237019
:10A130001B0A63700020F8BD0622EEE701232B8086
:10A14000F3681B782370F5E7F368002B16D008221C
:10A150002A801A8822701A88120A62705A88A2709D
:10A160005A88120AE2709A8822719A88120A6271D9
:10A17000DA88A271DB881B0AE371DBE72B80D9E761
:10A1800001202B80D7E7C04600D6FFFFF7B51600A9
:10A190000A781D0008AB1F880C000123022A18D181
:10A1A0004A685078117800022B4A08438018032827
:10A1B0000FD800F0E1FE02254439E06800F05CFFB2
:10A1C000C0B20723B84204D37B190193152B02DDDB
:10A1D0000D231800FEBDE0682A003100C01900F010
:10A1E00083FF6B4600209B88E268D0541B4B1B68A2
:10A1F000834203D01B68834200D098470023E8E7DE
:10A200000B23002FE5D1022DE2D1737832781B02A7
:10A210001343E2681380114B1B68002BEED01B68C0
:10A22000002BEBD00120E8E70B23002FD1D1062D26
:10A23000CED12A003100E06800F056FFDEE70B23A4
:10A24000002FC6D1012DC3D132787533012AC0D871
:10A25000E3681A70D2E7C04600D6FFFFF867FF1F19
:10A2600070B50C001500072837D800F085FE0414DF
:10A2700036361B36242E182015290BD8184E1622D8
:10A280000021300000F080FE22002900300000F0A4
:10A290002BFF002070BD18200229FBD11288114B22
:10A2A0001A80F6E718200829F4D10A000E48290080
:10A2B00000F062FFEDE718200129EBD10B4B10787D
:10A2C0000B49DA69FFF7DEFEE3E718200129E1D147
:10A2D000064B10780749DA6BF4E70220DAE7C0464C
:10A2E000E067FF1FC643FF1FBC43FF1F4C43FF1F18
:10A2F0007443FF1F9443FF1F030010B50020DB07CA
:10A3000004D50721024A034800F08CF810BDC0466E
:10A31000F8B700114C43FF1F054A030010680028DE
:10A3200003D082889A4201D1806870470068F6E7BE
:10A33000F069FF1F0A88030008009A4204D08A8847
:10A3400004309A4200D0002070470000F8B5F22295
:10A3500000230D4F0D4E796805004243337099423A
:10A3600000D07B600A4C0021200000F00DFE00238D
:10A370001A007C60AB4202D100203370F8BD01337B
:10A380002280DBB2F234F5E7E86AFF1FE66AFF1FBE
:10A39000F469FF1F73B56B4601900600684615000F
:10A3A0001980FCF779FF041E11D1002D0FD076899A
:10A3B000002E11D00C2000F0CFFE00280ED0084A4D
:10A3C0000460136886808560002B02D11060200035
:10A3D00076BD1A001B68F7E70224F8E71324F6E7B6
:10A3E000F069FF1F012100220A4B10B549420A4CB7
:10A3F000198099809A719A70084B207001201980F9
:10A400005A60FFF7A3FF2078FCF7A4FF0448FDF78C
:10A410005FFF10BD0068FF1FF06AFF1FE86AFF1FA3
:10A42000D1A40011022310B5002802D0FFF7B2FF1B
:10A430000300180010BD0000030010B50020DB076A
:10A4400004D50421024A0348FFF7A4FF10BDC0460B
:10A450000CB80011CC43FF1FF0B50E2687B0039354
:10A460000CAB1F8802ABF618050008003100029201
:10A47000FDF794F804000120002C0FD03088FFF77E
:10A480004BFF03000E20002B08D05E68002E05D085
:10A4900021002800039B029A0097B04707B0F0BD47
:10A4A0000A4B10B5984207D10122002352420A807C
:10A4B0008B708A808B7110BDFFF73CFF0028FAD0AB
:10A4C00001235B42038000238370F4E7FFFF000059
:10A4D000F8B5050001290AD1134E00243388F2276C
:10A4E000AB4219D028001149FFF7DAFF06E0022934
:10A4F00004D10139FDF76AFF0028EDD0F8BD3B001B
:10A5000063437268D018D35A002B09D03A00002157
:10A5100000F03AFD0134E4B2054B1B78A342EED8BB
:10A5200001235B423380DDE7E86AFF1F0068FF1FFD
:10A53000E66AFF1F10B5FFF7FDFE0300002083420F
:10A5400000D0987810BD0000F0B589B01C000EABAB
:10A5500080CB03901E8810AB1B78049202930B7A79
:10A560000D00DB0616D42B780593022B24D004981B
:10A57000FFF7D2FE002812D003689C46002B0ED0B5
:10A58000029B2200019329003B0064460398009639
:10A59000A04705E00498FFF7BFFE002802D10E2077
:10A5A00009B0F0BD8368002BF9D00A222900039876
:10A5B00098470028D7D0F3E76B6858781A786B4B28
:10A5C000000210439842D2D8043B984210D2684B04
:10A5D000984242D015D8674BC0180128C7D80B2025
:10A5E000002EDDD1EB681A7859683A80200028E007
:10A5F000614BC018032800D979E000F0BDFC846AE3
:10A60000789E5E4B9842B2D10B20002EC8D1012318
:10A610003B80EB6831001B7823706889013080B281
:10A62000FCF7BCFF3A88031E0ED0017802328A186C
:10A630003A80428962704289120AA270596802788F
:10A64000E01C00F051FD06E004323A8031000422A3
:10A65000601C00F099FC0020A2E70B20002E9FD187
:10A66000EB6807A91E8804233B80330A300026705C
:10A670006370FCF793FF051E28D004AB9A890E2364
:10A6800004A95B183E49C668FCF7FCFF00280BD103
:10A690002B783C486A680599FBF7B2FB002803D188
:10A6A000012304AA5B42D3813278022A06D1716861
:10A6B000201D00F019FD3B8802333B800E2304AAC5
:10A6C0009B181B88A3701B0AE370C4E704ABDE81F0
:10A6D000F4E70B20002E00D062E7E9680398FFF74B
:10A6E00029FF02233B802070000A6070B3E70B2033
:10A6F000002E00D054E70222EB681B883A802370BA
:10A700001B0A6370A7E7E86800F0B6FCC2B203005A
:10A710000720B24200D243E70DD00299DBB2711894
:10A72000994202DB921BD3B20293029BE9681A00A2
:10A730003B8089195AE70023F6E70B20002E00D052
:10A740002EE70722EB683A801A7822705A786270F6
:10A750005A88A2705A88120AE2701A792271DA882D
:10A760006271DB881B0AA37175E7C04604290000EB
:10A770000228000000D8FFFFFFD6FFFF03280000DB
:10A78000FFFF00003CB70011F0B58DB06B46002014
:10A79000089120229B5E83423DDAA64B187800F098
:10A7A000CBFE071E32D00378B02B2CD100790238B3
:10A7B00016281FD800F018FE17001E001E001E00ED
:10A7C00031001E0096001E001D011E0052011E00D9
:10A7D00073011E00CD011E0050021E001E001E004F
:10A7E0008E021E00E302944B94491B8878880B80EC
:10A7F000FBF746F83800FCF7C7FF914B1B68002BAE
:10A8000001D038009847380000F0E6FC8020089B13
:10A810000002434018000DB0F0BDEE220021874831
:10A8200000F0B2FB0BAA3B7B7989388900923A0091
:10A830000D32FCF7CBFD0400804B1B78002C3FD180
:10A8400046E0804B788805937F4B4100CB5A0BAE96
:10A85000073BDBB232880293002301937B4B21003C
:10A8600006930093059BFFF76FFE744D002810D1EF
:10A87000069B3A8A1B889A420BD138000599123000
:10A8800000F0BAFD002804D02B7862899B00EB18F9
:10A890005A80162306A81B18328820007989FCF7F5
:10A8A000F1FE2B7804009A00AA1851880029C3D021
:10A8B0000133DBB22B70002807D006A9C98A91802A
:10A8C000634A12889A42BCD802E001214942918031
:10A8D000002B04D059497888FBF706F88AE73E89AF
:10A8E0000A2479E000253E89574B06937B88069A17
:10A8F0005B009B5A033B9D4202DB002DF0D05BE0E6
:10A90000162206A812183B7B798900923A00300083
:10A910000D32FCF75BFD0590002858D04689017A7E
:10A920007888FCF71DFD041E44D1464B78880793B8
:10A93000069B4100C95A454B0439C9B206AAD28ABE
:10A9400006930291019400930599079BFFF7FCFD84
:10A95000041E2FD1069B39491A88931C002D26D13D
:10A960004B807988384B4900CB5A5119033B8B42B5
:10A9700020DD059B31485B8941190B71A91C01350C
:10A98000C9B2EDB2059145191B0A2B71059B2D49E2
:10A990000433181800F0A8FB2C4B059A1B88D31819
:10A9A000DDB22C4B9E4205D00136B6B29CE74988F9
:10A9B0009942D6D0002D0CD0204C2800618800F0A0
:10A9C000ABFB207021007888FAF79EFF12E7059C08
:10A9D000F0E7002C00D183E77B78142B00D109E746
:10A9E00016493B794E800B700C717888FAF73EFF60
:10A9F00000E7162406ABE41821003889FCF7CEFDE9
:10AA0000011E00D1B7E1788822880F4C45002C5BED
:10AA10000A4D013CE4B2029400240F4B01940095CE
:10AA2000FFF792FD041E00D014E129007888FAF7A0
:10AA30007BFFDFE6F06AFF1FB842FF1F0868FF1FB9
:10AA4000FC67FF1FFC68FF1F3864FF1FEC69FF1FD6
:10AA5000B642FF1FFFFF00000A68FF1F162406AB67
:10AA6000E41821003889FCF799FD011E00D182E12C
:10AA700078882288AE4C45002C5BAE4D013CE4B298
:10AA800002947C89AC4B01940095FFF75DFD041E98
:10AA900000D0DFE029007888FAF750FFAAE6002509
:10AAA000A44B1D803B00F6331B78A24A788807929E
:10AAB000AB4208D99E4B12880693069943005B5A15
:10AAC000013B9A4203DB0799FAF742FF92E616240C
:10AAD0006B00FB18059306ABE418059B2100188951
:10AAE000FCF75CFD011E03D1059B01241E8973E761
:10AAF0007888924B2288069C099343001B5B904EFA
:10AB0000013BDBB20293002300960193099BFFF700
:10AB10001BFD041E02D0059B1E895DE77B88069AFB
:10AB20005B009B5A079A108832881218934202DC05
:10AB30001B1A013B33807F4C02303288099900197F
:10AB400000F0D2FA2388328801359B182380EDB2B9
:10AB5000A8E70BAA3B7B7989388900923A000D322D
:10AB6000FCF734FC00250590059B002B04D10A243A
:10AB7000002D00D16EE060E0059B7888197AFCF723
:10AB8000EFFB0100041E63D1694C6C4B788806947E
:10AB90000993069B4400E45A694B063CE4B20BAEB1
:10ABA000328807930294019100930599099BFFF75E
:10ABB000CBFC041E4CD1079B5E491B881A1D002D3F
:10ABC00030D14A80059B5B4C5A8963191A716B1C02
:10ABD0009BB2E318120A1A71162306A832881B18B2
:10ABE00079890598FCF74EFDFF21AA1C2E1D03351F
:10ABF0000B00059092B2B6B2ADB2002803D006ABFE
:10AC0000DB8AD9B21B0AA218651911712B714C4D40
:10AC1000301D2A884949201800F066FA2B88F6185A
:10AC2000B5B2A1E74988914207D17A8806995200C6
:10AC3000525AEB18053A9A42C4DC3E4C280061880F
:10AC400000F0A2FA207021007888FAF78BFED1E597
:10AC5000002DF2D13E89BFE6162606ABF61831006C
:10AC60003889FCF79BFC3D000400FA3500282DD004
:10AC7000037A9B060CD400227B893989788800925C
:10AC80003A000C32FFF7E8FB041E10D03E8915E0B5
:10AC90003088FFF741FB00281AD08368002B17D0BB
:10ACA0002100122278889847041EE4D0EEE72B7822
:10ACB000002B02D17888FAF765FE00262B78002B4E
:10ACC00000D097E5002C00D194E585E60124DDE76E
:10ACD0000E24DBE7162506ABED1829003889FCF7B2
:10ACE0005DFC041E47D0037A9B0611D4154A7B886D
:10ACF0001188994203D01448814207D11380134B25
:10AD0000F2261D780023D9B2A94221D30924A1E754
:10AD10002888FFF701FB00282FD08368002B2CD058
:10AD20002100122278889847041EDFD092E7C0469F
:10AD30003864FF1F0868FF1F0A68FF1FFC68FF1FB9
:10AD4000EC69FF1FE86AFF1FFFFF0000E66AFF1FB4
:10AD500031005943546801336018615A0029D2D137
:10AD60003C0008342100F22200F0BEF9210078886E
:10AD7000FAF710FE3EE501246CE70E246AE71D4B4E
:10AD80001A887B889A4231D07888FAF70DFE31E52F
:10AD9000F223059851684343CD18C95A00291FD0A2
:10ADA0003B7A012B0BD16C88AB887888AA1D009464
:10ADB000FFF752FB041E02D000233B722E88F222C2
:10ADC0000021280000F0E0F800232B80059B0133D0
:10ADD000DBB20593084B05991B78064A8B42D7D8FE
:10ADE00001235B421380002CCED0F5E50026340011
:10ADF0000596EFE7E86AFF1FE66AFF1F70B50400DB
:10AE00000E001500FFF796FA031E08D13100054821
:10AE1000FFF790FA03001120002B02D01C800020C5
:10AE20009D7070BDFFFF0000F8B50B4F06003B782A
:10AE30000D001400FF2B0ED00A2000F06DFB011E48
:10AE400009D0B1230380002346800371C5800481AB
:10AE5000387800F029FAF8BD0D44FF1FF7B50F0050
:10AE600008A90600088809A90B240988002821D10F
:10AE70000234022B1ED1557813782D021D432B006E
:10AE80008B4301937334002B14D1FB6830001900FD
:10AE90000093FFF74FFB019C85420BD02A00300046
:10AEA0000099FFF7ABFF041E04D12A003000798916
:10AEB000FFF7BAFF2000FEBDF0B50E7885B0039015
:10AEC0000AA805880120022E0DD14C6827786478E5
:10AED00024023C43054FBC4205D10398DBB20196E6
:10AEE0000095FFF7BBFF05B0F0BDC046022900008A
:10AEF000034B10B51B68002B00D09847FEE7C046F7
:10AF0000F46AFF1F07B501A8FFF7F2FF044A0548DE
:10AF10000021121A00F0C8FAF8F7F4FBFEE7C04669
:10AF2000F86AFF1F1044FF1F01B40248844601BCA9
:10AF3000604700BF8939FF1F01B40248844601BC45
:10AF4000604700BFA136FF1F01B40248844601BC20
:10AF5000604700BFED4A010001B40248844601BCCD
:10AF6000604700BFC536FF1F01B40248844601BCDC
:10AF7000604700BFC926000001B40248844601BCF6
:10AF8000604700BF753BFF1F01B40248844601BC07
:10AF9000604700BF154D010001B40248844601BC62
:10AFA000604700BF5125000001B40248844601BC3F
:10AFB000604700BF5549010001B40248844601BC06
:10AFC000604700BF093AFF1F01B40248844601BC34
:10AFD000604700BF3D18000001B40248844601BC30
:10AFE000604700BF8D1BFF1F01B40248844601BCAF
:10AFF000604700BF1D3BFF1F01B40248844601BCEF
:10B00000604700BFC94A010001B40248844601BC40
:10B01000604700BF851F000001B40248844601BCA0
:10B02000604700BFDD66010001B40248844601BCF0
:10B03000604700BFA946010001B40248844601BC34
:10B04000604700BFADAE000001B40248844601BCB9
:10B05000604700BF613BFF1F01B40248844601BC4A
:10B06000604700BF8552010001B40248844601BC1C
:10B07000604700BFC521000001B40248844601BCFE
:10B08000604700BFDD52010001B40248844601BCA4
:10B09000604700BF9536FF1F01B40248844601BCDB
:10B0A000604700BFC51D000001B40248844601BCD2
:10B0B000604700BF2D2EFF1F01B40248844601BC2B
:10B0C000604700BFAD32FF1F01B40248844601BC97
:10B0D000604700BFD949010001B40248844601BC61
:10B0E000604700BF753AFF1F01B40248844601BCA7
:10B0F000604700BFE94C010001B40248844601BC2E
:10B10000604700BF9537FF1F01B40248844601BC69
:10B11000604700BF1147010001B40248844601BCEA
:10B12000604700BF350E000001B40248844601BCF0
:10B13000604700BF8530FF1F01B40248844601BC50
:10B14000604700BFE548000001B40248844601BCE6
:10B15000604700BF291C000001B40248844601BCBE
:10B16000604700BF3D4B010001B40248844601BC6A
:10B17000604700BF5522000001B40248844601BC6C
:10B18000604700BF810E000001B40248844601BC44
:10B19000604700BF090E000001B40248844601BCAC
:10B1A000604700BF6DBC000001B40248844601BC8A
:10B1B000604700BF2951010001B40248844601BC28
:10B1C000604700BFB352010001B40248844601BC8D
:10B1D000604700BF3119FF1F01B40248844601BC1B
:10B1E000604700BF434D010001B40248844601BCE2
:10B1F000604700BF5D34FF1F01B40248844601BCB4
:10B20000604700BFA54F010001B40248844601BC5D
:10B21000604700BF3555000001B40248844601BCB8
:10B22000604700BF0D31FF1F01B40248844601BCD6
:10B23000604700BF5D17000001B40248844601BCAE
:10B24000604700BF2526000001B40248844601BCC7
:10B25000604700BF8D12000001B40248844601BC63
:10B26000604700BF090E000001B40248844601BCDB
:10B27000604700BFF94C010001B40248844601BC9C
:10B28000604700BFC56D010001B40248844601BC9F
:10B29000604700BF691F000001B40248844601BC3A
:10B2A000604700BF7918000001B40248844601BC21
:10B2B000604700BF594F010001B40248844601BCF9
:10B2C000604700BF1D4B010001B40248844601BC29
:10B2D000604700BF5139FF1F01B40248844601BCDA
:10B2E000604700BF017F000001B40248844601BCF2
:10B2F000604700BF4551010001B40248844601BCCB
:10B30000604700BF056A000001B40248844601BCE2
:10B31000604700BF2124000001B40248844601BCFC
:10B32000604700BF4D1F000001B40248844601BCC5
:10B33000604700BFF30E000001B40248844601BC20
:10B34000604700BF453BFF1F01B40248844601BC73
:10B35000604700BF5147010001B40248844601BC68
:10B36000604700BF0D52010001B40248844601BC91
:10B37000604700BF055E000001B40248844601BC7E
:10B38000604700BF3533FF1F01B40248844601BC4B
:10B39000604700BF8B52010001B40248844601BCE3
:10B3A000604700BF091B000001B40248844601BC8D
:10B3B000604700BF0519FF1F01B40248844601BC65
:10B3C000604700BF456B010001B40248844601BCE0
:10B3D000604700BF4938FF1F01B40248844601BCE2
:10B3E000604700BFD532FF1F01B40248844601BC4C
:10B3F000604700BF893BFF1F01B40248844601BC7F
:10B40000604700BFCD4C010001B40248844601BC36
:10B41000604700BFE928000001B40248844601BC2F
:10B42000604700BF2146010001B40248844601BCC8
:10B43000604700BF75A9000001B40248844601BC02
:10B44000604700BFB14E000001B40248844601BC11
:10B45000604700BF311B000001B40248844601BCB4
:10B46000604700BFC939FF1F01B40248844601BCD0
:10B47000604700BF6D30FF1F01B40248844601BC25
:10B48000604700BFC9A9000001B40248844601BC5E
:10B49000604700BF014C010001B40248844601BC72
:10B4A000604700BF4550000001B40248844601BC1B
:10B4B000604700BFB70E000001B40248844601BCDB
:10B4C000604700BF5952010001B40248844601BCE4
:10B4D000604700BFF13AFF1F01B40248844601BC37
:10B4E000604700BF3520FF1F01B40248844601BCFD
:10B4F000604700BFE117000001B40248844601BC68
:10B50000604700BFEDA5000001B40248844601BCBD
:10B51000604700BFB54C010001B40248844601BC3D
:10B52000604700BF1D4D010001B40248844601BCC4
:10B53000604700BF156B010001B40248844601BC9E
:10B54000604700BFF54E010001B40248844601BCCB
:10B55000604700BF6571010001B40248844601BC28
:10B56000604700BF3D39FF1F01B40248844601BC5B
:10B57000604700BF0124000001B40248844601BCBA
:08B58000604700BFD91B000069
:10B588000200030004030503060307020803090376
:10B598000C030D001600090100000000E93A001133
:10B5A8001D3B00110000000002000000BAB50011A8
:10B5B800192A0F180A000000F1590000FD240000A4
:10B5C80041460100D9790011ED990011416E001131
:10B5D800DD7700114951001189A700111D4D001197
:10B5E800FD3F00112D41001100000000161600005B
:10B5F8000200000004B60011F4FFF3FFD2FC0000C3
:10B608006D4200110000000000000000444959008C
:10B6180042322E300030303230006769746875620B
:10B628002E636F6D2F70767678004B4559000000B9
:10B63800020000004CB60011292A282A272A262AA7
:10B64800252A242A0A180000050000000D501D00B4
:10B65800023CB40000011E00200000000900200088
:10B668003031323334353637383941424344454630
:10B678000000000001A00000000000006410B71DD9
:10B68800C8206E3BAC30D9269041DC76F4516B6B08
:10B698005861B24D3C7105502083B8ED44930FF0CA
:10B6A800E8A3D6D68CB361CBB0C2649BD4D2D38680
:10B6B80078E20AA01CF2BDBDFB349B5F80000080CD
:10B6C8000010000000000000435A0011CD70001166
:10B6D800675A0011D5740011EB5A0011AB740011B0
:10B6E800615B001181740011B35B00114976001190
:10B6F8001B5C0011497600114D5C001103760011A6
:10B70800615B001139740011D95B0011E1750011FA
:10B718000000000000000000BF5C0011E17500118E
:10B72800215D0011E5700011052A042A012A002A6A
:10B738000229032801280028011800180000000029
:10B748000000000000000000000000870101020165
:10B7580002010102010203030401030101010101C5
:10B768000303020103000D000E0010001100130076
:10B778001401070108010A010B011C011D02040242
:10B7880005020702080219021A021C021D0301031E
:10B79800020317000201000504000807000B0A0055
:10B7A8001716001D1C010201010504010E0D0111EF
:10B7B80010011413011716011A19020201020B0ACB
:10B7C800020E0D02111002141302171603050403CA
:10B7D8000807030B0A030E0D0001020307090A0BF1
:10B7E8000E0F101112141718191A1B1F20212200EE
:10B7F800D1A000118DA1001100000000020000007E
:10B8080042B7001100000000B9AE001100000000AE
:08B818000200000040B700111E
:020000041FFFDC
:1000000000000000653F0011C0B50011BCB5001133
:100010006061FF1F00000000000000000000000001
:1000200000000000000000000000000000000000D0
:1000300000000000000000000000000000000000C0
:1000400000000000000000000000000000000000B0
:1000500000000000000000000000000000000000A0
:100060000000000000000000000000000000000090
:100070000000000000000000000000000000000080
:100080000000000000000000000000000000000070
:100090000000000000000000000000000000000060
:1000A0000000000000000000000000000000000050
:1000B0000000000000000000000000000000000040
:1000C0000000000000000000000000000000000030
:1000D0000000000000000000000000000000000020
:1000E0000000000000000000000000000000000010
:1000F0000000000000000000000000000000000000
:1001000000000000000000000000000000000000EF
:1001100000000000000000000000000000000000DF
:1001200000000000000000000000000000000000CF
:1001300000000000000000000000000000000000BF
:1001400000000000000000000000000000000000AF
:10015000000000000000000000000000000000009F
:10016000000000000000000000000000000000008F
:10017000000000000000000000000000000000007F
:10018000000000000000000000000000000000006F
:10019000F932FF1F5931FF1FC16601000000000046
:1001A000000000000000000000000000000000004F
:1001B000000000000000000000000000000000003F
:1001C000000000000000000000000000000000002F
:1001D000000000000000000000000000000000001F
:1001E000000000000000000000000000000000000F
:1001F00000000000000000000000000000000000FF
:1002000000000000000000000000000000000000EE
:1002100000000000000000000000000000000000DE
:1002200000000000000000000000000000000000CE
:1002300000000000000000000000000000000000BE
:1002400000000000000000000000000000000000AE
:10025000000000000000000000000000000000009E
:10026000000000000000000000000000000000008E
:10027000000000000000000000000000000000007E
:10028000000000000000000000000000000000006E
:10029000000000000000000000000000000000005E
:1002A000000000000000000000000000000000004E
:1002B000000000000000000000000000000000003E
:1002C000000000000000000000000000000000002E
:1002D000000000000000000000000000000000001E
:1002E000000000000000000000000000000000000E
:1002F00000000000000000000000000000000000FE
:1003000000000000000000000000000000000000ED
:1003100000000000000000000000000000000000DD
:1003200000000000000000000000000000000000CD
:1003300000000000000000000000000000000000BD
:1003400000000000000000000000000000000000AD
:10035000000000000000000000000000000000009D
:10036000000000000000000000000000000000008D
:1003700005AF0011000000000000000000000000B8
:10038000000000000000000000000000000000006D
:10039000000000000000000000000000000000005D
:1003A0000000000000000000000000000D1BFF1F07
:1003B000000000000000000000000000000000003D
:1003C000000000000000000000000000000000002D
:1003D000000000000000000000000000000000001D
:1003E000000000000000000000000000000000000D
:1003F00000000000000000000000000000000000FD
:08183800006FFF1F4118FF1FA4
:10184000024981F3088802F08BFB0000006FFF1F44
:1018500070B500241E491F4A1F484C6308CA1B0567
:101860001B0DE4188242F9D11C4B80228B630021AE
:1018700009201B4B920519621A4B1B4DDA671B4B53
:10188000DA688243DA609A68194802409A60112047
:10189000296002F0B9F8112002F096F880226B6CF2
:1018A000112093436B64EE23DB006343114A1B0C4E
:1018B00013840122104B9A7401F004FC0F4B1B7827
:1018C000002B04D10E4B1021187802F081FB70BD63
:1018D000000005408805054000060540FF010000A6
:1018E00000F0004004E100E0003800403CF000401F
:1018F000FFDFFFFF1061FF1FC861FF1FFE63FF1FB7
:10190000FC61FF1F10B502F093F9072804D01228DC
:1019100008D0022808D010BD044A0420136B0133FC
:101920001363F8E70220F6E71420F4E7E064FF1FF2
:10193000F8B507000C0026002500503630785135E8
:10194000002804D10300287058342370F8BD29788A
:10195000CA00481E8141A3183800A25C5B68C9B266
:10196000FFF7D0FF00280DD12B78DA00A218013341
:1019700050602B703378044A013B3370136A013393
:101980001362D8E70123DFE7E064FF1F5C234343D2
:10199000074910B5C9180B0058331B78012B05D126
:1019A000FFF7C6FF034A936A0133936210BDC04636
:1019B0001465FF1FE064FF1F10B502F0F1FA064A3C
:1019C0000121130010CB4942D967044B136002F088
:1019D00057FA200010BDC04600E100E010001000E2
:1019E00010B5040002F0DCFA024B1C6002F048FA69
:1019F00010BDC04600E100E0431E5A425341A02200
:101A0000F0B5D2015B421340154D164A40019B18B8
:101A10002A18127E8BB00191002A1BD01A000832BE
:101A2000D46F0022E6B206AFE4B294420EDC28186E
:101A3000C369002B08D0019902AA117106AA049269
:101A400002AA167303A898470BB0F0BD1978B954D1
:101A50000132EAE71A7D1A7806AB01261A70E6E72A
:101A6000A067FF1F00400040F0B5254B0400400177
:101A7000C25C85B0002A2BD01A18117E002927D00D
:101A8000917E002924D01179022921D11689D78885
:101A9000D168F51BADB22A1C102D00D9102292B2CC
:101AA000BE4217D11818012303710023C269C380F5
:101AB00003819A4206D068460321037301710293A1
:101AC00001A890470820002C00D0192001F0FAFA54
:101AD00005B0F0BD013C65426C41A0256442ED01BA
:101AE0002C40084D1B186419074D0633013A92B279
:101AF000AA42EDD01888461C1E80085C2070F5E7CD
:101B0000A067FF1F00400040FFFF00000F220E4BA8
:101B100010B59868104002380A280BD802F02AF84D
:101B20000D0A0B0A0A110A0A0A0A060002210020FD
:101B3000FFF762FF10BD0121F9E70020FFF794FFD6
:101B4000F8E7DB6FF6E7C046004000400F220E4B7F
:101B500010B59868104002380A280BD802F00AF82D
:101B60000E0A0B0A0A120A0A0A0A060002210120BA
:101B7000FFF742FF10BD01210800F9E70120FFF740
:101B800073FFF7E7DB6FF5E70090004013B5334CC8
:101B90002378072B3DD8324B1A78324B002A39D1A3
:101BA0008022196852020A431A60252001F0ECFED7
:101BB00020232D4A11680B43802113606B460422B9
:101BC000C90508680733104228D080210422C905BE
:101BD000C86810422ED080212020C905CA688243DF
:101BE000CA6014221A701A78002A2FD18021C905E0
:101BF000C86820320243CA6014221A701A78002A78
:101C000028D11A4B1A7D22785A601D221A70593237
:101C1000DA6013BD1A6816490A40C5E7086802432E
:101C20000A6014221A701A78002ACED01A78013A63
:101C3000D2B2F7E7C8680243CA6014221A70197852
:101C40004A1ED2B21A700029F9D1C4E71A78013AB3
:101C5000D2B2C7E71A78013AD2B2CEE74843FF1FA3
:101C60001044FF1F3CF000404043FF1F0020004095
:101C7000FFFFFEFF564B70B51B68012B03D1554A81
:101C8000936D0133936502F0BBF9534B534A1860CF
:101C9000534B544C1A600123534A1360534A136048
:101CA0002378002B06D006225149524801F0E0FF6C
:101CB00000232370504A514B10681B78C1B2002B8F
:101CC0000ED14F4CC0B223785BB2002B4FDB237890
:101CD00024785BB264B21B0424021B191B18136026
:101CE0000B1C50294ED95023464A47491078DBB285
:101CF000FF2202284BD10868444C454D267890437A
:101D00002A78964254D9227824782E78023B5D10A6
:101D1000A31B6B435201D31A10335B1118430860A5
:101D200001F056FF031F012B45D83A4B1B78002BBF
:101D300006D0394B1B78002B02D0002001F0C0FFE9
:101D4000A122364B92009978354B4A431B689B1869
:101D5000832292009B181B78033B012B03D8AF20F2
:101D6000400002F09DF901222E4BDA8270BD2378EB
:101D700024785BB264B2FF33FF341B0424021B19C6
:101D80000138ABE7CAB2022AAED20223ACE7086838
:101D9000254C264D267890432A78964208D92278F9
:101DA00024782D78023B5B10641B63435201B2E739
:101DB0002378DBB2B2E70228D5D11D4B1B78013B5B
:101DC000022B03D91B4B1B78022BCCD16C20C8E70C
:101DD0009809FF1FFC0FFF1F2C64FF1FFF3F00002F
:101DE000141003403064FF1F0C1003400010034028
:101DF000D50BFF1F7211FF1FB40003408C09FF1F9A
:101E0000680AFF1F490AFF1F94000340460AFF1F8C
:101E1000470AFF1FF908FF1F2209FF1F300DFF1F90
:101E20003409FF1FBC0BFF1F440AFF1F450AFF1F99
:101E30001C09FF1F2309FF1F10B502F079F80022CB
:101E4000014B1A8010BDC0462864FF1F10B502F078
:101E50001FF9A121054A89009478054A6143126857
:101E6000044B5218528C1A8010BDC046300DFF1F13
:101E70003409FF1F2864FF1F10B50D4B0D4A9978D8
:101E8000A1239B004B431268D218531DD97F0A4BE4
:101E90001B88994209D2441C07D0C82805D0D269B2
:101EA0005B1A5A43054B5343C01801F0C1FF10BDE4
:101EB000300DFF1F3409FF1F2864FF1F710200004F
:101EC00070B5244D2B68002B28D002F071F82B68D8
:101ED000D8402B680400002B27D001F041FF2B686D
:101EE000D8401D4B1D4A9978A1239B004B43126893
:101EF000D118D25C91239B00002A20D0CA5801320D
:101F0000CA50174B17491B680868834214D3D23B49
:101F1000181A012A1AD0144B186070BD02F048F844
:101F2000124B196802F094F8D3E701F019FF0F4B38
:101F3000196802F08DF8D4E70D495B18E8E7CA503C
:101F40000C4B1B68DB68E418201AE4E7F530FF301F
:101F5000E1E7C0461C08FF1F300DFF1F3409FF1FBB
:101F60009C09FF1F2C64FF1FA009FF1F1808FF1FFB
:101F70002DFF3F003464FF1F70B504000D002829B9
:101F800016D10300A433C2881B889B1A0B4A9BB24C
:101F900093420DD906006A3605223100653001F002
:101FA00007FF002804D13100200001F029FE70BD98
:101FB0002900200001F004FFF9E7C046FE7F000081
:101FC000F8B50500012001F00BFE134CA36AA26ACC
:101FD0009342FBD1114E336001F01AFE1049030009
:101FE00008601048426894460F4A17680022BC45B2
:101FF00001D24268BA1A0D4802603268AD18A422B4
:10200000E562606A520302436262094A1278002A5A
:1020100001D00F3B0B60F8BD00F00040340AFF1FF9
:10202000E408FF1F28100040180AFF1F1C0AFF1FAA
:102030001C09FF1F70B580241025E405A3682B43FD
:10204000A36001F0EDFDA368AB43A36070BD000089
:10205000F7B5160080221C001023D205019191686B
:1020600005000B43936000225A4BD7301A6002F0F0
:102070001FF89D232A002F009B00EB58CA32012134
:102080000092FC37002B01D00021009A386801F043
:102090007FFE2900009BCB311A784F4BD3351A6055
:1020A0004B780A781B0213438A7812041A43CB78C0
:1020B0001B061343494A1BBA13604B790A791B026A
:1020C00013438A7912041A43CB7931001B06134358
:1020D000434A1BBA13606B782A781B021343AA7811
:1020E00012041A43EB781B0613433E4A1BBA1360D3
:1020F000019A330213433C4A13603C4B22001B1BE2
:102100009C4603293DDCB3089A0013005142B21AE1
:10211000032A46D1354AE018511A827840781204D1
:1021200000020243E05C043302430A600022FF2BFA
:102130004BDDF0222E4B12011A600F222D4B1A603C
:102140002D4A1368002BFCD00023224A2749136034
:10215000091B321D0B191B68043A180A23706070A2
:10216000180C1B0EA070E3700434002AF2DC8022ED
:1021700010213B68D20501333B6093688B43936029
:10218000F7BD6346D578981893782D061B042B432A
:10219000157804392B43557804322D022B43036004
:1021A000AFE7022A0AD1114AE05C511AE2185278CC
:1021B000120202430A6004339BB2B7E7012AB5D189
:1021C0000A4A521AE15C1160F5E7084959180A6099
:1021D0000433ACE7000004403C00044038000440F5
:1021E00034000440300004400C000440000104406E
:1021F000040004401000044014000440F7B515002A
:1022000080221C001023D2050091916807000B4327
:1022100093600023654AD730136001F049FF9D2386
:102220003E009B00F9583B00CA363200FC330029BF
:1022300000D07FE0586801F0ABFD390032785C4B8C
:10224000CB311A604B780A781B0213438A78AC466C
:1022500012041A43CB78281D1B061343554A1BBA98
:1022600013604B790A791B0213438A7912041A43CB
:10227000CB791B061343504A1BBA13604B7A0A7A78
:102280001B0213438A7A12041A43CB7A21001B06DD
:1022900013434A4A1BBA1360009A2B021343484A5D
:1022A00013602200474B1B1B0093009BCE785B18EA
:1022B00001938B7836061B0433430E78043833437E
:1022C0004E78043136023343019E33600328ECDC40
:1022D0000321A808431C9B002940800003292BD11F
:1022E0003849E5185E18A9786D78E35C09042D0279
:1022F000294319433160030008330021FF2B2DDDF2
:10230000314B324919600F21314B196001232749A4
:102310000B60304B19680029FCD006211B680B406C
:10232000042B20D080220020D20593680A318B43F1
:102330009360FEBD01217DE7022908D121495D1886
:10234000E1184978E35C090219432960D3E70129C0
:10235000D3D11C495918E35C0B60CCE71948181815
:1023600001600433CAE7002310490B606346002B69
:102370000CDC3B00FC335A68102101325A60802289
:10238000D205936801208B439360D2E7009B9B1892
:102390001B68190A13705170190C1B0ED37004239B
:1023A0005B4291709C440432E0E7C0460000044068
:1023B0003C00044038000440340004403000044035
:1023C0000C0004400001044004000440080F000019
:1023D000100004401400044070B5061E19D00222FB
:1023E0005A4B9B799343012B13D1594B1A78FF2AEF
:1023F0000FD15A78FF2A0CD19A78FF2A09D1DA78BE
:10240000FF2A06D11A79FF2A03D15B79FF2B00D16D
:1024100099E0504B0C201A78012A08D000224E4D2A
:102420001A7029780B00093B042B01D8212070BDBC
:102430004B1F012BFAD9454CA37B042B00D982E01A
:10244000A279032A00D97EE09A1ED2B2012A02D8CC
:1024500060881F2877D9002E56D0012E73D1A0880E
:102460000128E3D0002907D1581E032803D801F022
:1024700081FB121715122E702978481E032811D8D7
:102480000025364B1D602823237501F089FCA842E6
:1024900027D0A580CAE702212970EDE70421FBE7D8
:1024A0000321F9E707390129C0D82D490968C96A0C
:1024B0008906BBD52B4908780028B7D1012A01D954
:1024C000002BB3D102230B708021274D26338901C5
:1024D0002878237501F0A4FD80212878890101F076
:1024E00077FD0123A380214B1B78002B0AD0FA2211
:1024F00080211F4B92001B8809025A431A4B1878FF
:1025000001F09EFC002092E701F04AFD2B78A680A6
:10251000073B012B03D917482E7001F019FD114B11
:10252000114C1A78002A06D08021002220788901D7
:102530001A7001F075FD01F0A3FC802120780902DA
:1025400001F06EFDDEE7122071E7C046A60BFF1F0B
:102550006B09FF1F1A09FF1F1C09FF1F4809FF1FF6
:102560003464FF1F2309FF1F1B09FF1F2109FF1FE1
:102570002C09FF1F0010004010B5002901D001F008
:10258000C7FC10BDF7B5604B01919978A1239B0062
:102590004B435E4A060014681022E418D6235B0001
:1025A000E0583623FF33E35C00279343222B41D1CD
:1025B000574B0F3A1A600760012501F0F9FA019BA9
:1025C0001880E8235B00E35C002B01D0B34258DDA8
:1025D0000023504FFB70AD33FF33E3581A68002AD5
:1025E00003D09B88DB439B071DD03823FF33E35C7C
:1025F000002B18D09B235B00E35C002B13D1D1335D
:10260000FF33E35CB3420EDAA4235B00E15AE01827
:10261000090A023101F024FB23000122FE33013EAE
:1026200001351A87FA70E8235B00E35C002B2AD09F
:10263000A8B2FEBD03683D00002BBED081880430E7
:10264000090A023101F00CFBD6235B00E3581F603E
:10265000B2E72300B133BA00FF33985801378188BD
:102660000430090A023101F0FBFAE8235B00E35C65
:10267000BB42EEDCE822F61AED1800235200A35408
:10268000A6E70027F1E7200001F0FAFA00281FD0A2
:10269000002E1DDD7319882647190193B60020000E
:1026A00001F06EFB5A3080002018406801358188A7
:1026B0000430090A023101F0D3FA200001F068FC6D
:1026C000A3590133A351BD4202D0019B9D42E6D1E3
:1026D000114BE35C002BABD095239B00E35C002BFC
:1026E000A6D00E4BE15A0029A2D00D4AA35C994214
:1026F00002D90133A3549BE700231A212000A354DD
:1027000001F09EFC94E7C046300DFF1F3409FF1F07
:1027100000140340E010FF1F5A0200007202000084
:102720005E0200000D4970B54A6E0D4CD2038B69F4
:10273000D20BA24206D80B4D0224AA4204D901F0C2
:102740001FFC70BD02246442E21815007E2425405F
:102750002242F4D0A3432B438B61F0E700F000400A
:102760000A200000FC1C0000F8B51D4B1D4F1A7814
:10277000002A10D1BA7B002A02D101321A7003E07C
:10278000032AFAD0022AF8D001F00AFB0022012025
:10279000154B1A70F8BD154B154D1C68154B9E78DE
:1027A00001232B702878C0B200F09EFBBB7B002B6E
:1027B0000BD101F07DFAA1239B007343E41883231E
:1027C0009B00E41823782B70E4E7032B02D101F07F
:1027D00067FBF0E70020022BDCD101F0B9FAEAE751
:1027E0001C09FF1FA60BFF1F2309FF1F3409FF1F32
:1027F000490AFF1F300DFF1FF0B587B00EAD2F78CF
:102800000FAD2D780593AC46634614000E4D0CAA0F
:1028100012782E7803930D9B009201932200059B62
:10282000029701F0E5FB2E70012C01D0042C08D199
:10283000802206498B889343054A1278D2011343BC
:102840008B8007B0F0BDC0461C09FF1F6C11FF1F35
:102850007809FF1F0B001B3B70B504003020E02BF4
:102860000DD81300E025493BFF3B9BB2ED00AB4286
:1028700005D8034B200019825A8201F021FB70BD5C
:102880008410FF1F10B501F0BBFB054B00205B68F7
:10289000052B04D9034A5268D20200D4980810BD0F
:1028A00000100040FCE100E070B501F079FB0D4B39
:1028B0001B68FC33DC691D6AFFF7E4FF641984427E
:1028C00004D2094B01241B68002B07D004220024EA
:1028D000064B1A70064A93690133936101F0D0FAEE
:1028E000200070BD3464FF1F9809FF1F2309FF1FDC
:1028F000FC0FFF1F70B50C4D2B68FC335C6A01F0B8
:102900004FFBFFF7BFFF2B680025FC339B6AE318E2
:10291000834204D2054B1B68AB4200D1051B01F07A
:10292000AFFA280070BDC0463464FF1F9809FF1F2E
:10293000D722044B92009B5810B5002B00D098472B
:1029400010BDC0460000FF1F10B501F0FBF8FFF7F7
:10295000EFFF2749274BCA6D274C1A4084235B00A1
:102960001343CB65254B1B68186A01F039F9244BDA
:10297000244A1A60244B254A1A60A022244B520094
:102980001A60244B187801F0BBF92000224901F0AD
:1029900077FB0023A3600233A360204B2049236010
:1029A00003232048A36001F06BFB10221E4BFF2085
:1029B0001A60802252031A60802292031A608022D9
:1029C00012041A6001F07CF9012001F029FAFA20C2
:1029D000400001F05DF9582001F062FB134801F05E
:1029E00087F9012001F06CFB072001F031F910BDDF
:1029F00000F0004000FEFEFF141000403464FF1F92
:102A0000000003400180063DBC0003403408000084
:102A1000A40003404A0AFF1F71020000C30900001E
:102A2000FFFF3F002810004000E100E0307500008B
:102A3000674E336888331B6883F3088801F048F9D0
:102A4000644A6549136800200B401360634B644A75
:102A50001B68934200D1A6E001F00AFB0221614A03
:102A600013688B431360FFF76FFF5F4B5F4C187861
:102A7000C0B201F045FA0023A3600233A3605C4BAF
:102A80000120236001F0ACF80323A36001F0D0FA29
:102A9000040001F0B5FA050001F0CAFA554B1860C0
:102AA00001F0DEF9544B1968621A531EA14200D29C
:102AB00013008022D203934201D39B029B0A326807
:102AC000D16AC90700D471E04C491C0C09689BB25B
:102AD0004C4359432402090A641803264849FC322E
:102AE00093680A6847489B1A474A0768126847492B
:102AF0009B18474A9A1833409208DB190A60036012
:102B0000042B03D9013233400A6003600E68414947
:102B1000A619300001F09CFA3F4F3E493B68C318AC
:102B20003B603000019301F073F93C4E30680818A7
:102B300038493060884205D9019B01333B6001F080
:102B400067F9316001F0FCF8354B1B78002B0DD094
:102B500001F056FA334B621B196812188A4232D2BE
:102B60004919091B091A304801F08AFA2F4E337AA5
:102B7000002B0ED001F044FA621BF168121891424A
:102B800024D94919091B091A294801F079FA0023A7
:102B90003372284B83F3088801F0C2F9002001F05A
:102BA00067FA01F01DF901F063FA5CE7DC019900B6
:102BB0000234641A5900641A09214B438033CB4014
:102BC000A408E41889E7FA218900CCE71A49DBE771
:102BD0003464FF1F1CF00040FFFFC1FF0C0AFF1F01
:102BE000B641210310000040490AFF1F14100040A5
:102BF000C3090000100AFF1F340AFF1F380AFF1F15
:102C0000200AFF1F280AFF1F1C0AFF1F240AFF1F9C
:102C1000C4090000710200006008FF1F2C0AFF1F9A
:102C20001C09FF1FE408FF1F00100040740BFF1F6A
:102C30003C10004000000020DC050000A022054BF5
:102C400092009B5810B5002B01D0984710BD01F0A1
:102C50002FF9FBE70000FF1FA122054B92009B58B4
:102C600010B5002B01D0984710BD01F021F9FBE70A
:102C70000000FF1FA222054B92009B5810B5002BAD
:102C800001D0984710BD01F013F9FBE70000FF1FCA
:102C9000A322054B92009B5810B5002B01D09847FA
:102CA00010BD01F005F9FBE70000FF1FA422054B52
:102CB00092009B5810B5002B01D0984710BD01F031
:102CC000F7F8FBE70000FF1F70B501F099F94F4BD3
:102CD000186000F075FF0400C30702D400F0B0FFD5
:102CE00070BD00224A4B1A604A4B187801380428FC
:102CF00029D800F03FFF0320181C2400200001F019
:102D000037F80128ECD0444C2378042B6ED100F026
:102D10006FFF0028E4D001F07BF9582001F0C0F9E2
:102D200002232370DCE7200001F052F8E9E72000DD
:102D300001F096F9E5E7200000F0D2FFE1E720007E
:102D400000F0EEFFDDE700F043FF0500012808D1A9
:102D5000324B1B78053B012B03D82000FFF76EFF99
:102D6000D1E72D4B1B78022B01D0052B20D1022D52
:102D700028D12B4B9B7BAB431CD12000FFF76CFF72
:102D8000264B18780128BED16405BCD424492522DD
:102D90004B7B034205D1233A13405A425341263319
:102DA0001A000B7D9342AED9322001F061F8AAE7F8
:102DB000022D07D1194B1B78052B11D12000FFF7ED
:102DC00059FFDDE7012D0BD1012B03D12000FFF7C7
:102DD0005FFF98E7062B03D12000FFF767FF92E71C
:102DE000200001F065F8022D8DD1C9E7032B04D135
:102DF0000C4B987C00F0D4FE72E7072B00D06FE7F5
:102E0000094B987B00F0F4FF6AE7C0469C09FF1F5E
:102E10009809FF1F9009FF1F2309FF1F1C09FF1FAF
:102E2000A60BFF1FBC0BFF1FD40BFF1FFA210A4B81
:102E30000A4A49001A640A4A5A500A4A04395A503E
:102E4000094A08319A64094A5A50094A5C315A5071
:102E5000084ADA667047C0460000FF1FF927FF1FC7
:102E6000F528FF1FA928FF1FD923FF1F6927FF1F70
:102E7000791EFF1F4D1EFF1FF7B50B0CFF27012208
:102E8000009300233C001E001D009446019089B26F
:102E900062469A401000084018413618B6B2FF2F1B
:102EA00002D1012E00D19FB2009802401A41AD1804
:102EB000ADB2FF2C02D1012D00D19CB20133102BF9
:102EC000E6D10320012E07D1012D04D1019B24015D
:102ED000E4191C700138FEBD102EFCD10238102DF3
:102EE000F9D00230F7E700008023F7B59C46264B67
:102EF000264F01932649274A274D284C284B022864
:102F00001AD1604638600868264E30408026360365
:102F10003043086001990978002909D11660224AD6
:102F20002A60224A2260E02219689143A03A1BE0FD
:102F30008021C9021160F2E766463E600F68194EB3
:102F40003E408027FF023E430E6001990978002928
:102F50000DD1176001280ED1154A2A60154A22604A
:102F6000E02219689143C03A0A431A60F7BD8021F4
:102F700089021160EEE7E0210F4A02432A600F4AFE
:102F800022601A688A43F0E74B0AFF1FE000034003
:102F9000D80003409000034000000340500003406D
:102FA00040000340FFFFE3FF0280063D804508220A
:102FB0000180063D80660822008006988055082220
:102FC000F8B51E4B80261A680020140034403242A7
:102FD00032D11A681A4F32431A6001223B68063018
:102FE00093433B6000F0FCFD0122164D2B681E430D
:102FF0002E603B680A2613433B608027BF00124BBC
:103000001B683B4211D1013EF6B2FF2E09D17E2250
:103010000E4B1C682B68E40B1440934323432B6036
:1030200005E0082000F0DCFDE9E7002EEFD180226A
:103030002B68600893432B60F8BDC046C4F0004085
:103040005CF0004018F0004068F0004060F0004084
:1030500010B500F04DFF01215820034A00F068FE32
:10306000FFF7AEFF10BDC046600AFF1F10B5782203
:103070000021034800F0ECFE00F032FF002010BDFC
:103080002867FF1F70B5040000F08AFF00230C20A2
:103090000B4A010059438D18515C00290DD0A14203
:1030A00008D1012300246B7000F012FF00F0E8FE4D
:1030B000200070BD01330A2BEBD11224F6E7C04685
:1030C0002867FF1F70B5040000F06AFF0023190095
:1030D0001D000D4A1078002806D0A0420CD1557072
:1030E00001310C320A29F5D1002B0AD100F0F8FE8B
:1030F00000F0C6FE002070BD5078461EB0411B187F
:10310000EEE700F0E5FEF3E72867FF1FF7B50400E0
:103110000C20002384460E4D019267465F43E85D14
:103120007E19A04212D000280BD10A4B9C46624661
:103130001B7808331370019B70707C557160B3600D
:10314000FEBD01330A2BE8D10320F9E70720F7E79A
:103150002867FF1F2467FF1F8020F8B5484BC00574
:103160001B68C1248360474BFF251A680123134362
:103170004361454BA4001A68444B40211A60444BFC
:103180001A68444B1A60444B1A59AA431A51C52273
:1031900092009E58AE433143802699509F583F4934
:1031A000F6010F403E439E509E5880273602360A55
:1031B0003043985080201A5900020A4002431A51A5
:1031C00004341A59364E3F04324080263A431A518D
:1031D0001A5936061202120A32431A5108341A5981
:1031E00080260A4002431A51C32292009F58B446D7
:1031F000AF4337439F509F58294E0F4007439F507E
:103200009F58374080263604374380269F509F586A
:1032100036063F023F0A37439F50C0221F59AF4333
:103220003A431A511A591202120A1643C6221E5163
:1032300092009C58AC4365462C439C509C580025FA
:103240000C4020439850C72080001A58154C11405C
:10325000C02212020A431A50134B1B78DB08AB4200
:1032600001DC0020F8BD2378002B06D0A368002BDA
:1032700000D0984701350C34EEE71220F2E7C04643
:103280004443FF1F4043FF1FB0F000402067FF1F73
:10329000B4F000401C67FF1F00E100E0FF00FFFFEB
:1032A000FFFF00FF2867FF1F2467FF1F030010B503
:1032B0001F2809D8072200201340072404490A7850
:1032C000A24313430B7010BD00230620F5E7C04650
:1032D0002467FF1F054B06491B780A6805485B07F2
:1032E00002401B0B134300200B6070472467FF1F35
:1032F0001CF00040FFFFC1FF70B50C25FFF7EAFF8F
:103300000A4B1C780A4BE4086543ED18002C01D1E8
:10331000200070BD2B78002B06D06B68002B00D0EE
:103320009847013C0C3DF1E71220F2E72467FF1FAC
:103330001C67FF1F70B50D00040000F031FE402136
:103340000F4AAD00136865198B431360AC4208D176
:10335000002202200B4B1A600B4B186000F098FD06
:10336000FEE7637801212078002B00D0032100F0D4
:1033700027FE6178207800F093FC0434E6E7C0462D
:103380001CF00040C4F00040C0F000401FB5002118
:1033900002220B0001910091052000F0E9FD0223BB
:1033A0000B490A681A42FCD120230393039B5A1E3F
:1033B0000392002BFAD1074A1368002BFCDA0B2486
:1033C0006C442000012100F00BFE207804B010BDF9
:1033D00090C8004000C8004013B504000A4B019398
:1033E000019B002B01D1112016BDFFF7CFFF230059
:1033F0000340044205D0052000F0F2FB019B013B95
:10340000EDE71800F0E7C046FFFFFF0707B500F043
:10341000C7FD80220821D205936A0191002B01D1BA
:103420000739916202210C4A11600199481E0190EE
:103430000029FAD103311160053101910199481E2B
:1034400001900029FAD11160002B02D18022D2050F
:10345000936200F015FD07BD00C00040F0B52D4C93
:1034600089B02378002B4FD1FEF7A6FA02232A4F0A
:1034700003903A681A42FCD120230693069B5A1EF9
:103480000692002BFAD1254E3368002BFCDA01207E
:10349000FFF7A2FF011E02D0112009B0F0BD03000A
:1034A00003220190009005AD9F2000F061FD0321F3
:1034B000280000F095FD02233A681A42FCD120232F
:1034C0000793079B5A1E0792002BFAD13368002BF3
:1034D000FCDA0120FFF780FF0028DDD10398FEF71A
:1034E0007FFAAA786B7811041B020B4329780B43EF
:1034F00063601300113B0A49052B07D80123934051
:10350000A3600B60012323700020C6E780231B0308
:10351000F6E7C0462C43FF1F90C8004000C800409B
:103520009808FF1F1E4B30B55A6818781D4B85B0A0
:10353000D31859424B4101210093002300F060FC55
:10354000194B1A4A02259A6300221A6510325A65ED
:103550008022C4219D65164B1648D202DA67890085
:103560004258154B80241A4080231B0413434350B8
:10357000642341200393E40500F006FA402000F0A4
:1035800003FA6562039D6B1E0393002DFAD103239A
:103590006362FFF73BFFA562FFF760FF05B030BD38
:1035A0003843FF1F95FFFEF700C80040050001FFEC
:1035B00004E100E000E100E0FFFF00FFF0B585B0AE
:1035C0000700FEF7F9F9022305002D4C22681A4284
:1035D000FCD120230093009B5A1E0092002BFAD1AD
:1035E000284E3368002BFCDA0120FFF7F5FE002897
:1035F00003D01124200005B0F0BD234B236002232B
:1036000022681A42FCD120230193019B5A1E019289
:10361000002BFAD13368002BFCDA0120FFF7DCFE27
:103620000028E6D1194B1F60022322681A42FCD100
:1036300020230293029B5A1E0292002BFAD1336878
:10364000002BFCDA0120FFF7C7FE0028D1D1104B78
:103650002360022322681A42FCD120230393039B98
:103660005A1E0392002BFAD13368002BFCDA01209A
:10367000FFF7B2FE041EBCD12800FEF7B1F9B9E78E
:1036800090C8004000C8004001000006A8C80040E3
:103690000180000110B50020FFF790FF10BD000071
:1036A00010B5064B18705960FFF73CFF002113203E
:1036B000034AFFF72BFD002010BDC0463843FF1F13
:1036C0002535FF1FF0B5040085B003920291FEF787
:1036D00073F9882263035B0B52051A438023DB05D1
:1036E0009D6A8023274F0092BA68002601901B0331
:1036F0009A420CD9F82326001B041E401C4206D017
:103700008022214B52025E6219680A431A60002D22
:103710000BD100F045FC02221C4B1A608023DB0514
:103720005A62013A9A6200F0ABFB0023039A93427B
:1037300020D1002D0AD100F033FC144B03221D6070
:103740008023DB055A629D6200F09AFB8023BA68F1
:103750001B039A4208D9002E06D000220A4B0C49BE
:103760005A621A680A401A600198FEF739F9002077
:1037700005B0F0BD009A0299D2181278CA540133EC
:10378000D4E7C0462C43FF1F00C8004000C00040E3
:10379000FFFFFEFFF0B587B0029103920400FEF731
:1037A0000BF9019000F0FCFB802302250122234E3F
:1037B000DB0535605D629A6200F062FB204F3B687A
:1037C0002B42FCD120230493049B5A1E0492002B0D
:1037D000FAD11C4D2B68002BFCDA0120FFF7FCFD11
:1037E000002802D0112007B0F0BD2000039A0299F2
:1037F00000F08EFA022304003A681A42FCD120231A
:103800000593059B5A1E0592002BFAD12B68002BBD
:10381000FCDA0120FFF7E0FD051EE3D100F0C0FB5C
:1038200080230322DB0535605A629D6200F028FB8D
:103830000198FEF7D5F8E0B2D5E7C04600C00040D9
:1038400090C8004000C80040F0B5802489B0060050
:10385000FEF7B2F8E405A36A02250393029000F094
:103860009FFB0123304F3D606562A36200F008FBBF
:103870002E4C23682B42FCD120230593059B5A1E16
:103880000592002BFAD12A4D2B68002BFCDA01207F
:10389000FFF7A2FD002803D01124200009B0F0BDDD
:1038A000244B2360022322681A42FCD12023069372
:1038B000069B5A1E0692002BFAD12B68002BFCDACD
:1038C0000120FFF789FD021EE6D11B4B03211E607C
:1038D000030001900090202000F04AFB02232268A0
:1038E0001A42FCD120230793079B5A1E0792002BF4
:1038F000FAD12B68002BFCDA0320FFF76DFD041EC4
:10390000CAD100F04DFB80230322DB053C605A62E4
:103910009C6200F0B5FA039B002B01D1FFF776FD06
:103920000298FEF75DF8B8E700C0004090C800407C
:1039300000C800400100000694C8004007B500021E
:1039400001910422000A01A9FFF724FF0EBD000027
:1039500073B5050005240B4AA3005B429B18196848
:103960006B46DE1D3000FFF787FA022804D133785A
:103970002B55013CEFD276BD052CFCD00128FAD1A5
:103980000230F8E7140900111F2807D8012380220C
:103990008340D20591680B43936070473F2808D855
:1039A0000123802220388340D20551690B435361A3
:1039B000F3E75F28F1D80123802240388340D20505
:1039C000116A0B431362E8E71F2807D80122802100
:1039D0008240C9058B6893438B6070473F2808D8A5
:1039E0000122802120388240C9054B6993434B61F5
:1039F000F3E75F28F1D80122802140388240C905D1
:103A00000B6A93430B62E8E71F2810D8802302005B
:103A1000DB05153A1968012A06D82022914319605E
:103A200019680A431A60704701228240F6E73F286E
:103A300011D880230200DB05353AD968032A06D85D
:103A400010229143D960D9680A43DA60EBE701227A
:103A500020388240F5E75F28E5D842238022181AF3
:103A6000413B8340D205516A99435162516A0B43ED
:103A70005362D8E710B50400012813D1A0221849D9
:103A800092050B685B015B0913430B60154B164AEB
:103A900019681140154A0A431A60402219680A43FE
:103AA0001A6010BD0028FCD101000A2000F048FA7D
:103AB00021000B2000F044FAC0220A4B9200196842
:103AC0000A4340211A601A688A431A60B0220449E6
:103AD00012060B685B015B0913430B60E1E7C0460C
:103AE00014F000401CF000407F00FEFF80FD01004C
:103AF00072B6074A1368013313600422054B1A603B
:103B00000023054A13608022D2055360FEE7C046B9
:103B10007808FF1FC0F00040C4F0004005490B6862
:103B2000002B05D1044A0A6004490A60044A136064
:103B30007047C046140AFF1F841E0000380AFF1F8A
:103B4000C4F000400023034A1360034A1360034A91
:103B50001360704754F0004040F1004044F10040D1
:103B600002B4714649084900095649008E4402BC16
:103B70007047C04602B4714649084900095C4900D3
:103B80008E4402BC7047C04603B4714649084000E9
:103B90004900095A49008E4403BC704700000000E8
:103BA00001B40248844601BC604700BF4DF90000E3
:103BB00001B40248844601BC604700BFCD0C01003F
:103BC00001B40248844601BC604700BFBD0B010040
:103BD00001B40248844601BC604700BFDD0C01000F
:103BE00001B40248844601BC604700BF018900005F
:103BF00001B40248844601BC604700BF01D7000001
:103C000001B40248844601BC604700BF85C1000082
:103C100001B40248844601BC604700BFBD5C01009E
:103C200001B40248844601BC604700BFDD3F00008C
:103C300001B40248844601BC604700BFE927000088
:103C400001B40248844601BC604700BFDD0A0100A0
:103C500001B40248844601BC604700BFF90D010071
:103C600001B40248844601BC604700BFC115010091
:103C700001B40248844601BC604700BFE94C010022
:103C800001B40248844601BC604700BF71B0000027
:103C900001B40248844601BC604700BF85120100A0
:103CA00001B40248844601BC604700BFB5B20000C1
:103CB00001B40248844601BC604700BFE9F6000039
:103CC00001B40248844601BC604700BFED6B0100AF
:103CD00001B40248844601BC604700BFC9A9000086
:103CE00001B40248844601BC604700BFF5350100BD
:103CF00001B40248844601BC604700BF8D11010039
:103D000001B40248844601BC604700BFEDA5000035
:103D100001B40248844601BC604700BF95730100AE
:103D200001B40248844601BC604700BFF935010078
:103D300001B40248844601BC604700BF016701002E
:103D400001B40248844601BC604700BFD54401006D
:103D500001B40248844601BC604700BF19FA000064
:103D600001B40248844601BC604700BF6D0B0100EE
:103D700001B40248844601BC604700BF0134010021
:103D800001B40248844601BC604700BFD9B00000BE
:103D900001B40248844601BC604700BF21440000D2
:103DA00001B40248844601BC604700BFA9D80000A6
:103DB00001B40248844601BC604700BFCD4C0100FD
:103DC00001B40248844601BC604700BF51B80000FE
:103DD00001B40248844601BC604700BF09340100B9
:103DE00001B40248844601BC604700BF855201000F
:103DF00001B40248844601BC604700BFC1F700001F
:103E000001B40248844601BC604700BFC56D010093
:103E100001B40248844601BC604700BF090E00009F
:103E200001B40248844601BC604700BF691101002B
:103E300001B40248844601BC604700BF89370100D5
:103E400001B40248844601BC604700BF8B520100A8
:103E500001B40248844601BC604700BFB70E0000B1
:103E600001B40248844601BC604700BFC16601003E
:103E700001B40248844601BC604700BF61370100BD
:103E800001B40248844601BC604700BF9DA9000000
:103E900001B40248844601BC604700BFA1AF0000E6
:103EA00001B40248844601BC604700BF75F80000B9
:103EB00001B40248844601BC604700BFE917010015
:103EC00001B40248844601BC604700BF116E000087
:103ED00001B40248844601BC604700BF21A900002C
:103EE00001B40248844601BC604700BFADAE00008B
:103EF00001B40248844601BC604700BFED68010080
:103F000001B40248844601BC604700BF8914010027
:103F100001B40248844601BC604700BFE9D40000F8
:103F200001B40248844601BC604700BF7997000095
:103F300001B40248844601BC604700BF8D82000086
:103F400001B40248844601BC604700BF9D9B00113C
:103F500001B40248844601BC604700BFC1A500000F
:103F600001B40248844601BC604700BF0DAF001198
:103F700001B40248844601BC604700BF496D01009E
:103F800001B40248844601BC604700BFD1AE0000C6
:103F900001B40248844601BC604700BF5976010065
:103FA00001B40248844601BC604700BF75A9000007
:103FB00001B40248844601BC604700BFE90B010020
:103FC00001B40248844601BC604700BF49B200000A
:103FD00001B40248844601BC604700BF0D52010095
:103FE00001B40248844601BC604700BF3D71010036
:103FF00001B40248844601BC604700BF9D6A0000CE
:1040000001B40248844601BC604700BFC95C01009E
:1040100001B40248844601BC604700BF6DF6000051
:1040200001B40248844601BC604700BFB35201009E
:1040300001B40248844601BC604700BF156B010013
:1040400001B40248844601BC604700BF53B9000078
:1040500001B40248844601BC604700BF090E00005D
:1040600001B40248844601BC604700BF053401002A
:1040700001B40248844601BC604700BF016C0100E6
:1040800001B40248844601BC604700BF2D6C0100AA
:1040900001B40248844601BC604700BFF9ED00004E
:1040A00001B40248844601BC604700BF7912010098
:1040B00001B40248844601BC604700BF8944000047
:1040C00001B40248844601BC604700BFE51201000C
:1040D000020000003EB7001101000000B0B5001161
:1040E000020000003AB70011010000001041FF1F5C
:1040F00002000000B8B5001101000000C461FF1FFC
:104100000200000038B70011030000003461FF1FF7
:1041100012000000020000003EB700110100000084
:10412000F8B50011020000003AB7001101000000CC
:10413000F5B500110200000002B6001103000000F6
:104140008F61FF1F0200000038B70011030000005C
:10415000A461FF1F020000003AB700110100000037
:10416000F4B500110200000000B6001103000000C9
:104170006561FF1F0200000038B700110300000056
:104180008661FF1F020000003EB700110100000021
:1041900038B60011020000003AB70011010000001B
:1041A0005942FF1F020000004AB600110100000042
:1041B00032B60011020000003AB700110100000001
:1041C0005842FF1F0200000048B600110100000025
:1041D000AC61FF1F020000003AB7001101000000AF
:1041E0005742FF1F0200000046B600110100000008
:1041F00022B60011020000003AB7001101000000D1
:104200005642FF1F0200000044B6001101000000EA
:104210001DB60011020000003AB7001101000000B5
:104220005542FF1F0200000042B6001101000000CD
:1042300018B60011020000003AB70011010000009A
:104240005442FF1F0200000040B6001101000000B0
:1042500014B60011020202020202000035490011E8
:10426000F948001168B6001190011D0018001800EF
:10427000FFFF07010203040506020106000000001B
:10428000000000000000000000000000000000002E
:10429000000000000000000003000000000100001A
:1042A00000000111FFFF00005048593600000000D7
:1042B000000000000B000500F0000000B400002822
:1042C000002800283075A000A000A000A000000871
:1042D0000008E001F00010001000100010001000B5
:1042E000100050005000500010001000D0070000D7
:1042F000000000000F0001000500307507001000ED
:10430000010081FF00000000FF000000A56D00110A
:10431000AD6B00113D690011FFFF0100FF000000BF
:10432000C19700113D950011559400110000000047
:104330000000000000000800040000003B0001082D
:104340005902E00188212800FF000000020000005F
:104350003EB700110100000004B800110200000087
:104360003AB7001101000000C943FF1F020000001E
:1043700036B7001101000000E067FF1F02000000D7
:104380003AB7001101000000C843FF1F02000000FF
:1043900034B7001101000000C643FF1F02000000F7
:1043A0003AB7001101000000C443FF1F02000000E3
:1043B00032B7001101000000BC43FF1F18001800B5
:1043C0001D00900102000003020200000200000034
:1043D0003EB700110100000018B8001102000000F3
:1043E0003AB70011010000000C44FF1F020000005A
:1043F00030B70011000000000000000002000000C3
:0E44000038B70011030000000068FF1F20FF06
:040000051FFF184180
:00000001FF
